:020000041000EA
:1000000000B5324B212058609868022188439860DF
:10001000D860186158612E4B002199600221596106
:100020000121F02299502B49196001219960352056
:1000300000F044F80222904214D00621196600F024
:1000400034F8196E01211966002018661A6600F04E
:100050002CF8196E196E196E052000F02FF8012189
:100060000842F9D1002199601B49196000215960AB
:100070001A491B48016001219960EB211966A021F2
:10008000196600F012F800219960164914480160C1
:100090000121996001BC002800D000471248134993
:1000A000086003C880F30888084703B5996A0420EC
:1000B0000142FBD001200142F8D103BD02B5186610
:1000C0001866FFF7F2FF186E186E02BD00000240BE
:1000D000000000180000070000035F00212200005C
:1000E000F4000018222000A00001001008ED00E03C
:1000F00000000000000000000000000074B24E7A12
:1001000000200420F7010010C3010010C5010010F9
:10011000C1010010C1010010C1010010C101001097
:10012000C1010010C1010010C1010010C701001081
:10013000C1010010C1010010C9010010CB01001065
:10014000CD010010CD010010CD010010CD01001037
:10015000CD010010CD010010CD010010CD01001027
:10016000CD010010CD010010CD010010CD01001017
:10017000CD010010CD010010CD010010CD01001007
:10018000CD010010CD010010CD010010CD010010F7
:10019000CD010010CD010010CD010010CD010010E7
:1001A000CD010010CD010010CD010010CD010010D7
:1001B000CD010010CD010010CD010010CD010010C7
:1001C00000BE00BE00BE00BE00BE00BE00F04BF888
:1001D000103800BEF2EB8871F4AE001018AF0010BA
:1001E0003402001090A31AE700202149086006C8D5
:1001F00081F3088810471F48006800282FD10DA4FC
:100200000ECC002902D000F012F8F9E71A491B4A77
:10021000002000E001C19142FCD1194988471949E9
:1002200088471949884700BEFDE701C901C29A42C3
:10023000FBD3704718AF0010C00000204805002015
:10024000A0B300100000042000000420A0B30010A0
:1002500000100420001004200000000070470B482C
:1002600004F068FF0047EFF30580C0B2704700005C
:1002700008ED00E0000000D000800020A48E0220E5
:1002800061360010911F00101D36001057560000F7
:1002900006005250ABB36053D4A500100600525074
:1002A000861C0302E4A50010060052505422A29DB1
:1002B000F4A5001005005250DE65F468A0B30010EC
:1002C000F8B5C04610B5064C2378002B07D1054B76
:1002D000002B02D0044800E000BF0123237010BDB2
:1002E000088102200000000038950010044B10B572
:1002F000002B03D00349044800E000BF10BDC046F6
:10030000000000000C8102203895001070B5012318
:10031000964A1370964A12689340A020C0059549EA
:1003200043509301A021C9058C466344DB68DB017F
:10033000F7D4914B1A680123934008008D4943502C
:100340009301A021C9058C466344DB68DB01F7D427
:100350008A4B1A6801239340080086494350930151
:10036000A021C9058C466344DB68DB01F7D4844BCC
:10037000196801238B4060467E4A83508B01A0227E
:10038000D20594466344DA6880235B0414001C4061
:100390001A42F3D17B4D2A68303280239B011343EC
:1003A00001221A600021072003F06AFB2A68764BBD
:1003B00018680430754B9A4200D0082400190021B7
:1003C00003F05EFB7249072003F09CFB684B1A6840
:1003D000704B0C2A00D9A9E06F490B40D20213439D
:1003E0000C229343043A13436C4A13406C4A134063
:1003F0006C4A1340012213436B490B4093435C4A00
:1004000010688201A021C9058C4662440021116058
:1004100051609160136108F0FDFD574B1A685D4B08
:100420000C2A00D988E05C490B40D20213430C220D
:100430009343043A1343594A1340594A1340594AC3
:1004400013400122134358490B4093434A4A106812
:100450008201A021C9058C466244002111605160CF
:100460009160136108F0D6FD444B1A68494B0C2A81
:1004700068D849490B40D20213430C229343043AF3
:100480001343464A1340464A1340464A134001224A
:10049000134345490B409343384A10688201A02119
:1004A000C9058C466244002111605160916013615E
:1004B00008F0B0FD324B1A68364B0C2A48D8364942
:1004C0000B40D20213430C229343043A1343334AA2
:1004D0001340334A1340334A134001242343324A22
:1004E0001340A343264A10688201A021C9058C4607
:1004F00062440021116051609160136108F08AFD2F
:10050000204B1868204B196803688C40A343036094
:1005100008F030FE254B1B78002B1FD0244B1A68A7
:10052000184B1868234908F06FFE70BD224B234A10
:10053000C021234803F076F81F4B204AC0212048F1
:1005400003F070F81C4B1D4AC0211D4803F06AF8E7
:10055000194B1A4AC0211A4803F064F8144B1A6860
:10056000084B1868174908F04FFEDEE7948E02200A
:100570006C870220440400007087022074870220E8
:1005800078870220D4860220548E0220000020505A
:100590000D03001010801F00FF87FFFF3FF8FFFFD3
:1005A000FFFFBFFFFFFFDFFFFFFF7FFF9E8E0220E9
:1005B000D08602209096001038950010B09600105A
:1005C000589500107096001070B501239C4A137066
:1005D0009C4A12689340A020C0059B494350930158
:1005E000A021C9058C466344DB68DB01F7D4974B37
:1005F0001A68012393400800934943509301A021B6
:10060000C9058C466344DB68DB01F7D4904B1A685C
:100610000123934008008C4943509301A021C90550
:100620008C466344DB68DB01F7D48A4B19680123ED
:100630008B406046844A83508B01A022D2059446A9
:100640006344DA6880235B0414001C401A42F3D12F
:10065000814D2A68303280239B01134301221A60A6
:100660000021072003F00CFA2A687C4B186804303C
:100670007B4B9A4200D008240019002103F000FAB5
:100680007849072003F03EFA6E4B1A68764B0C2A25
:1006900000D9BCE075490B40D20213430C229343AE
:1006A000043A1343724A1340724A1340724A134089
:1006B0000122134371490B409343624A106882013F
:1006C000A021C9058C4662440021116051609160EF
:1006D000136108F09FFC5D4B1A68634B0C2A00D92C
:1006E0009BE062490B40D20213430C229343043A2D
:1006F00013435F4A13405F4A13405F4A134001228D
:1007000013435E490B409343504A10688201A02175
:10071000C9058C46624400211160516091601361EB
:1007200008F078FC4A4B1A684F4B0C2A00D97AE043
:100730004E490B40D20213430C229343043A134315
:100740004B4A13404B4A13404B4A13400122134378
:100750004A490B4093433E4A10688201A021C905D3
:100760008C4662440021116051609160136108F071
:1007700051FC384B1A683C4B0C2A5AD83B490B4069
:10078000D20213430C229343043A1343384A1340D2
:10079000384A1340384A134001242343374A134050
:1007A000A3432C4A10688201A021C9058C466244EB
:1007B0000021116051609160136108F02BFC264DFF
:1007C0002868264B1968036822008A409343036017
:1007D00008F0D0FC2A4B1A6828682A4908F014FD52
:1007E000294D2868294E036832689440A34303606A
:1007F0000022316808F052FD3168286808F0BAFC20
:10080000234B1A682868234908F0FEFC70BD224B70
:10081000224AC021224802F005FF1F4B1F4AC02177
:100820001F4802F0FFFE1C4B1C4AC0211C4802F06E
:10083000F9FE194B194AC021194802F0F3FEC046CF
:10084000948E02206C8702204404000070870220EE
:100850007487022078870220D4860220548E0220DA
:1008600000002050C905001010801F00FF87FFFF07
:100870003FF8FFFFFFFFBFFFFFFFDFFFFFFF7FFF2F
:10088000D086022050960010788E0220588E0220CA
:10089000748E02203C04002038950010B0960010A1
:1008A0005895001070B501239B4A13709B4A12683B
:1008B0009340A020C0059A4943509301A021C90547
:1008C0008C466344DB68DB01F7D4964B1A6801233E
:1008D00093400800924943509301A021C9058C46DA
:1008E0006344DB68DB01F7D48F4B1A680123934024
:1008F00008008B4943509301A021C9058C466344ED
:10090000DB68DB01F7D4894B196801238B40604613
:10091000834A83508B01A022D20594466344DA684F
:1009200080235B0414001C401A42F3D1804D2A68D6
:10093000303280239B01134301221A6000210720DB
:1009400003F09EF82A687B4B186804307A4B9A4271
:1009500000D008240019002103F092F877490720FD
:1009600003F0D0F86D4B1A68754B0C2A00D9BBE028
:1009700074490B40D20213430C229343043A1343AD
:10098000714A1340714A1340714A134001221343C4
:1009900070490B409343614A10688201A021C90548
:1009A0008C4662440021116051609160136108F02F
:1009B00031FB5C4B1A68624B0C2A00D99AE0614902
:1009C0000B40D20213430C229343043A13435E4A72
:1009D00013405E4A13405E4A1340012213435D49AF
:1009E0000B4093434F4A10688201A021C9058C46F1
:1009F00062440021116051609160136108F00AFBAC
:100A0000494B1A684E4B0C2A00D979E04D490B40EE
:100A1000D20213430C229343043A13434A4A13402D
:100A20004A4A13404A4A13400122134349490B40A2
:100A300093433D4A10688201A021C9058C46624457
:100A40000021116051609160136108F0E3FA374BA7
:100A50001A683B4B0C2A59D83A490B40D20213432F
:100A60000C229343043A1343374A1340374A134046
:100A7000374A134001242343364A1340A3432B4AE9
:100A800010688201A021C9058C46624400211160D2
:100A900051609160136108F0BDFA254D2868254B1F
:100AA0001968036822008A409343036008F062FBE0
:100AB000294B1A682949286808F0A6FB2868284E9F
:100AC000036832689440A34303600022316808F051
:100AD000E5FB3168286808F04DFB224B1A6828684E
:100AE000214908F091FB70BD204B214AC0212148CB
:100AF00002F098FD1D4B1E4AC0211E4802F092FDD7
:100B00001A4B1B4AC0211B4802F08CFD174B184A98
:100B1000C021184802F086FD948E02206C870220C6
:100B20004404000070870220748702207887022026
:100B3000D4860220548E022000002050A508001008
:100B400010801F00FF87FFFF3FF8FFFFFFFFBFFF81
:100B5000FFFFDFFFFFFF7FFFD086022030960010EF
:100B6000588E0220748E0220200400203895001038
:100B7000B09600105895001070B5040001238B400A
:100B8000DDB2013DEDB2FF20002307E080214901E5
:100B900019435A00084E91530133DBB21F2B09D879
:100BA0002A001A40A242F1D05A0003490348505289
:100BB0001800F1E770BDC04624810220A0A0FFFF0D
:100BC000F8B5012008F02EFAC84C2060012008F08A
:100BD00029FAC74B1860012008F024FAC54B1860A9
:100BE000012008F01FFAC44B18602168C34A0C2981
:100BF00000D92AE1C24B1A40C9020A430C208243A1
:100C000008210A43BF4B1A40BF4B1A40BF4B1A4042
:100C100001231A43BE4B1A4010239A43130020228B
:100C2000134383430B43B24A12680C2A00D912E1E2
:100C3000B3491940D3020B43B64A1068B64A12684A
:100C40000432B649884200D10BE1082152183F2AEC
:100C500000D908E1B2491940D3030B43A94A134014
:100C6000F822D2001343A24A1068A4490C2800D9E4
:100C7000FFE0A34A1140C00201430C24A143082015
:100C80000143A04A1140A04A1140A04A114001224C
:100C900011439F4A1140102291430A0020210A4328
:100CA000A2430243934909680C2900D9E7E094481C
:100CB0001040CA02024397490C68974909680431F9
:100CC0009648844200D1E0E0082009183F2900D965
:100CD000DDE093481040CA0302438A490A40F821E4
:100CE000C9000A4383490C6884480C2C00D9D4E01D
:100CF00083490840E40220430C25A84308242043EC
:100D00008049084080490840804908400121084343
:100D10007F49084010218843010020200143A94356
:100D20002143754800680C2800D9BCE0744C0C4085
:100D3000C102214377480568774800680430774C42
:100D4000A54200D1B5E0082400193F2800D9B2E03F
:100D5000734C0C40C10321436A480140F820C00095
:100D6000014365480568654C0C2D00D9A9E064482D
:100D70000440ED022C430C26B44308252C43614863
:100D80000440614804406148044001200443604835
:100D9000044010208443200020242043B0432843F3
:100DA000524C24680C2C00D991E0554D0540E002CE
:100DB0002843584C2668584C24680434574DAE429A
:100DC00000D18AE0082564193F2C00D987E0544DF2
:100DD0000540E00328434B4C2040F824E400204326
:100DE000454C27684B4C26684B4C24680834A500BA
:100DF0007519BF01A024E405A44667443D60494C31
:100E00007C608026B601BE6038613A480068800187
:100E100060440560444FE7194760866001613449CA
:100E20000968890161440D604048201848608E605F
:100E30000A612E4A12689201624415603C498C4650
:100E4000644454609660D360F8BD3A4B3A4AC0217E
:100E50003A4802F0E7FB374B374AB831374802F0DF
:100E6000E1FB0021F2E6364B364AB221334802F06C
:100E7000D9FB304B304AC021304802F0D3FB2D4B18
:100E80002D4AC0212D4802F0CDFB00201DE72C4B40
:100E90002C4AB221294802F0C5FB264B264AC02124
:100EA000264802F0BFFB234B234AC021234802F00F
:100EB000B9FB002448E7224B224AB2211F4802F026
:100EC000B1FB1C4B1C4AC0211C4802F0ABFB194B68
:100ED000194AC021194802F0A5FB002573E7184BF9
:100EE000184AB221154802F09DFBC0466C870220CB
:100EF00070870220748702207887022010801F00EC
:100F0000FF87FFFF3FF8FFFFFFFFBFFFFFFFDFFF90
:100F1000FFFF7FFFD4860220548E02200000205065
:100F2000FF7FE0FF000002200080FFFF0000FFFFC6
:100F30000080FEFF38950010B09600105895001004
:100F4000A4950010CC96001010B50D4B1B78002B0B
:100F50000CD1EFF3108472B60A4B1B78002B06D02D
:100F6000012B07D0022B08D084F3108810BDFFF7A7
:100F7000CDF9F9E7FFF796FCF6E7FFF725FBF3E776
:100F8000948E02209D8E0220F0B5DE4657464E46D6
:100F90004546E0B595B002900D00140003931EABDA
:100FA0001E781FAB1A78934620AB1F7821AB1A88A6
:100FB00090460A1980231B029A4200D30DE23D4B52
:100FC000984200D911E2182E00D910E25A460F2A91
:100FD00000D90EE2052F00D90DE2002F00D10CE25E
:100FE000BB18102B01DD0020F8E1802292020021C5
:100FF000314805F04DF8314B1D60314B1C60314BD1
:101000001E70314B01221A700023039806E0C25C67
:101010002E49895C2E4AD1540133DBB2B342F6D358
:101020002A4B5A469B5C1A0003932A4B1A700520E0
:1010300002F0ACFC04F05CFF8146029B580004F017
:1010400057FF011C484604F034FF8146224D234BD4
:101050001D60280008F004F9214B9B4621481860C8
:1010600008F0FEF85B461B68AB420ED0072100205B
:1010700001F0B8F8194B1A68174B9A4207D00721AC
:10108000012001F0AFF8002508E00621EFE7062176
:10109000F6E7062101F0A6F80135EDB2B54223D2FC
:1010A0000E4B1A680A4B585D0B4B9A42F1D0072140
:1010B000F0E7C04600E1F50500800020A08B02208B
:1010C0009C8B02209C8E02209B8E0220E4960010B6
:1010D000848B0220A08E022000002050D4860220A3
:1010E000788E022000003050C54D0121286808F09C
:1010F00051F80200C34B9A461860286853009B18A9
:10110000DB00D033C318802149010B43802109063D
:101110001960196003680432012191400B43036098
:10112000B94908F055F8B94B9B4618605346196801
:101130002868002300931D33022208F0E9F85B467B
:101140001B689A461022002108A804F0A1FF802500
:101150006D020895F8235B0209938023DB020A9352
:10116000C0231B030A93102208A904A804F096FFC9
:101170005346191D5A1D059B0293A54B0298034027
:10118000C9010B43120313430593102204A90CA8B1
:1011900004F084FF0F9B02939E4B029A13401D4361
:1011A0000F95484604F0CCFE85B2002D00D110E129
:1011B000280004F09DFE011C484604F070FE8721C3
:1011C000C90504F08CFE04F0BBFEC3B21B022D0463
:1011D0001D430C950E9B02938F4A1A408F4B13436D
:1011E0000E930D9B02938E4A1A4080235B04134397
:1011F0000D93834D2A681100303180239B011943E0
:10120000012008602D32FF321343802252001A6001
:101210008449063002F04CFC0121072002F030FC2A
:101220002A68784B186804307F4B9A4200D1D2E08C
:101230000823C018012102F023FC744B1A68714B7B
:101240009A466F4B9B460CAB51460968584600685E
:1012500008F096F8754D0121286807F09BFF744B44
:10126000994618602A6843001B18DB00D033D31856
:10127000802149010B438021090619601960136818
:101280000430012181400B4313604346D8B239003A
:10129000FFF772FC6749286807F09AFF664B98468B
:1012A00018604B461968286801230093002208F053
:1012B0002FF84B4619682868002300933B00039ED3
:1012C000320008F025F843461F681022002108A8C4
:1012D00004F0DEFE80256D020895F8235B02099379
:1012E0008023DB020A93C0231B030A93102208A960
:1012F00004A804F0D3FE3B001F331A00059B0293A1
:10130000434B02990B40FF013B43120313430593E8
:1013100007990291CA00D208802189050A430792E1
:10132000464A13400593102204A910A804F0B6FE03
:10133000102210A90CA804F0B1FE0F9B0293354BAC
:1013400002990B40F6031E430F963D4B1E4080232F
:10135000DB041E430F963B4B1E400F960C95FFF788
:101360002FFC5B461A6853461D6811680123AB4089
:1013700099430B431360013C51682800103001234E
:1013800083400B42F8D1291D89008C5051680B42D3
:10139000FCD10435AD0001235B42AB50264B1A68EB
:1013A000234C224D0CAB2168286807F0E9FF29681F
:1013B00020680A68012383409A4313430B6000238B
:1013C000214A1370214A1370214B02221A70012006
:1013D00004E00023FAE600232BE7002015B0F0BC60
:1013E000BB46B246A946A046F0BD0020F6E7002065
:1013F000F4E70020F2E70020F0E70020EEE7C04627
:10140000D4860220548E022050960010D0860220EE
:101410007F00FEFFFF7FF0FFFFFF0AFE0000D1010B
:10142000FFFFFFE0C905001000002050788E022069
:10143000588E02203C040020748E0220FFFFFF9F84
:101440001FFCFFE3FF83FFFF948E0220958E022096
:101450009D8E0220F0B5DE4657464E464546E0B525
:1014600095B002900D00140003931EAB1E781FABC5
:101470001A78934620AB1F7821AB1A8890460A1938
:1014800080231B029A4200D301E23A4B984200D9D2
:1014900005E2182E00D904E25A460F2A00D902E2CA
:1014A000102F00D901E2002F00D100E2BB18102B51
:1014B00001DD0020ECE18022920200212E4804F0A0
:1014C000E7FD2E4B1D602E4B1C602E4B1E702E4BCD
:1014D00001221A700023039806E0C25C2B49895C44
:1014E0002B4AD1540133DBB2B342F6D3274B5A46D1
:1014F0009B5C1A000393274B1A70052002F046FAF2
:1015000004F0F6FC8146029B580004F0F1FC011C3B
:10151000484604F0CEFC81461F4B9B461F4D1D6084
:10152000280007F09DFE5B461B68AB420ED00721EA
:10153000002000F057FE184B1A68184B9A4207D04B
:101540000721012000F04EFE002508E00621EFE70C
:101550000621F6E7062100F045FE0135EDB2B54261
:101560001ED20D4B1A680A4B585D0C4B9A42F1D0B3
:101570000721F0E700E1F50500800020A08B0220A4
:101580009C8B02209C8E02209B8E0220E4960010F1
:10159000848B0220A08E0220D486022000002050DE
:1015A000C44D0121286807F0F5FD0200C24B9A46A0
:1015B0001860286853009B18DB00D033C3188021C3
:1015C00049010B4380210906196019600368043240
:1015D000012191400B430360B84907F0F9FDB84B76
:1015E0009B461860534619682868002300931D33F2
:1015F000022207F08DFE5B461B689A4610220021EE
:1016000008A804F045FD80256D020895F8235B02CB
:1016100009938023DB020A93C0231B030A93102241
:1016200008A904A804F03AFD5346591D9A1D059BCC
:101630000293A44B02980340C9010B4312031343C6
:101640000593102204A90CA804F028FD0F9B029317
:101650009D4B029A13401D430F95484604F070FCC1
:1016600085B2002D00D10EE1280004F041FC011CE0
:10167000484604F014FC8721C90504F030FC04F04E
:101680005FFCC3B21B022D041D430C950E9B0293FD
:101690008E4A1A408E4B13430E930D9B02938D4A34
:1016A0001A4080235B0413430D93824D2A68110076
:1016B000303180239B011943012008602D32FF3215
:1016C0001343802252001A608349063002F0F0F979
:1016D0000121072002F0D4F92A68774B18680430FA
:1016E0007E4B9A4200D1D0E00823C018012102F0BD
:1016F000C7F9734B1A68704B9A466E4D0CAB514646
:101700000968286807F03CFE0121286807F042FDBF
:101710000200734B99461860286853009B18DB0041
:10172000D033C318802149010B4380210906196079
:10173000196003680432012191400B430360694B37
:101740003B43694A5381694907F042FD684B9B4618
:1017500018604B461968286801230093002207F09F
:10176000D7FD4B4619682868002300933B00039E71
:10177000320007F0CDFD5B461F681022002108A84B
:1017800004F086FC80235B029B460893F8235B02EF
:1017900009938023DB020A93C0231B030A931022C0
:1017A00008A904A804F07AFC3B0008331A00059B42
:1017B0000293444B02990B40F9010B43120313436C
:1017C0000593102204A910A804F068FC102210A9A7
:1017D0000CA804F063FC0F9B02933B4B02990B4057
:1017E000F6031E430F96434B1E408023DB041E432B
:1017F0000F965B460C930E9B0293344B029A134058
:101800000E934B4619680CAB3A00286807F0B8FDF8
:10181000FFF7D6F92A6853461D6811680123AB40CB
:1018200099430B431360013C516828001030012399
:1018300083400B42F8D1291D89008C5051680B421E
:10184000FCD10435AD0001235B42AB50244B1C6836
:1018500011680123A34099430B4313605168200092
:101860001030012383400B42F8D10434A4004346D6
:10187000A3500023204A1370204A1370204B0122EA
:101880001A70012004E00023FCE600232DE700206D
:1018900015B0F0BCBB46B246A946A046F0BD00203C
:1018A000F6E70020F4E70020F2E70020F0E7002050
:1018B000EEE7C046D4860220548E022030960010F7
:1018C000D08602207F00FEFFFF7FF0FFFFFF0AFEB1
:1018D0000000D101FFFFFFE0A5080010000020502C
:1018E000588E0220406000002804002020040020C0
:1018F000748E02201FFCFFE3948E0220958E02203E
:101900009D8E0220F0B5D6464F464646C0B590B0F3
:1019100082460F0016001C0018AB1D7819AB1B780F
:1019200099461AAB1B7898468A1880231B029A4264
:1019300000D36AE1B94B984200D96DE1182D01D965
:10194000002063E1802292020021B54804F0A0FB50
:10195000B44B1F60B44B1E60B44B1D70B44B424679
:101960001A70B44B00221A70002106E0635CB24A80
:10197000D25CB24B5A540131C9B2A942F6D3AE4B34
:101980004A469B5C9946AE4B4A461A70052001F0C8
:10199000FDFF04F0ADFA041C5346580004F0A8FA09
:1019A000011C201C04F085FA071CA64CA6482060E8
:1019B00007F056FC0121206807F0ECFB0200A34B66
:1019C0001860206853009B18DB00D033C3188021B7
:1019D00049010B438021090619601960036804322C
:1019E000012191400B4303604346002B18D09849D6
:1019F00007F0EEFB974B1860944B1968914C2068E8
:101A0000002300932033002207F082FC22688E4BD3
:101A10009A420BD00721484600F0E4FB00240CE07A
:101A20008D4907F0D5FB8B4B1860E5E70621F2E7FF
:101A3000062100F0D7FB0134E4B2AC4208D2814B5E
:101A40001A687E4B185D804B9A42F1D00721F0E76F
:101A50004346002B00D1AAE07E4B1C6810220021D7
:101A600008A804F015FB80235B020893F8235B02AF
:101A700009938023DB020A93C0231B030A931022DD
:101A800008A904A804F00AFB22000A32059B03936C
:101A9000724B03990B40E401234312031343059354
:101AA000102204A90CA804F0F9FA0F9B03936C4BC5
:101AB000039A13400F93381C04F042FA84B2002CAE
:101AC00000D19EE0200004F013FA011C381C04F041
:101AD000E6F98721C90504F002FA04F031FAC0B230
:101AE0000002240404430C940E9B03935D4A1A40A5
:101AF000A023DB0213430E930D9B03935A4B039ACF
:101B000013404A46120613430D934E4C22681100AF
:101B1000303180239B011943012008602D32FF32B0
:101B20001343802252001A605049063001F0C0FF72
:101B30000121072001F0A4FF2268444B18680430FB
:101B4000414B9A425FD00823C018012101F098FF51
:101B5000404B1A683D4C3B4D0CAB2168286807F0A0
:101B60000FFCFFF72DF8296825680A680123AB40B0
:101B70009A4313430B60013E48682C001034012344
:101B8000A3400342F8D12A1D920056504A681342DE
:101B9000FCD10435AD0001235B426B500023344A75
:101BA0001370344A1370344A137001202EE0294B0D
:101BB0001C681022002108A804F06AFA80235B0246
:101BC0000893F8235B0209938023DB020A93C02366
:101BD0001B030A93102208A904A804F05FFA221D2F
:101BE0000534059B03931D4B03990B40D20113430E
:101BF000240323430593102204A90CA804F04EFAF1
:101C000053E700206CE700239EE7002010B0E0BC03
:101C1000BA46B146A846F0BD0020F7E700E1F50559
:101C200000800020A08B02209C8B02209C8E022032
:101C30009E8E02209B8E0220E4960010848B022050
:101C40009F8E0220D486022000002050548E022055
:101C500070960010D0860220909600107F00FEFF44
:101C6000FF7FF0FFFFFF0AFEFFFFFFE00D03001004
:101C7000948E0220958E02209D8E0220024B1878B1
:101C800001235840C0B27047948E0220F0B5CE4672
:101C9000474680B580468C46434B1B78002B10D0BE
:101CA000424B1B68424A12689B1842461360414BE4
:101CB00062461B6813604048C0BCB946B046F0BDE0
:101CC00001338022120293421CDA9A003A4C1259D4
:101CD0000132F5D1013B17D4344A1568344A1268F1
:101CE000AD186A1E9A4211D95B1B344A91464B4487
:101CF000304A13602F4B1C68314B1B78002B2CD1C2
:101D0000002143E00023E7E72C4BE5E75B1B0133B1
:101D1000284A1360EEE72B4B9A5D023A0123934069
:101D20000340921BD3401F430136274B1B78B3421D
:101D3000F1DC631CA400204AA750802212029342C7
:101D400009D21C0001318D422AD9A3001A4A9858A1
:101D500000260027E9E70024F4E70021F3E7194B08
:101D60009E5C0123B3400340B61AF3401F43013287
:101D7000154B1B789342F2DC631CA4000E4AA7505B
:101D800080221202934209D21C0001318D4207D9F0
:101D9000A300094A985800220027E9E70024F4E745
:101DA000014B01221A707BE7958E0220A08B022046
:101DB0009C8B0220A48B022000800020FF7F00006B
:101DC0009B8E0220848B02209C8E022070B584B0F2
:101DD000002004F005FB431C1FD063490A78531C04
:101DE000DBB20B7061498854012B10D0022B16D046
:101DF000022B12D91C009A1E5C498A5CAA2A0CD1BB
:101E00005A1E8A5C552A08D10022002118E00A785F
:101E1000552AEBD0544B00221A7004B070BD534ABF
:101E20005278AA2AE4D0504B00221A70F5E701320A
:101E30004E4DAE5C0138FF387040685401310132BC
:101E4000944206DD4948805CF028F0D0474D685444
:101E5000F4E7464A9278002A08D0012A10D0444874
:101E600004F07CFA404B00221A70D6E7052B03D011
:101E70003F4804F073FAF5E73E4804F06FFAF1E7E3
:101E80003D4B3E4A13601B78012B27D0022B46D0D6
:101E9000364C6579230009332B22A15CE26A1202D9
:101EA0000A432721605CA16A090201432320265CC2
:101EB000606A000230436E1EB54102952579019596
:101EC0002125645D0094FFF71DFD002848D02C48B3
:101ED00004F044FA2B4B01221A70C3E72A4B1C0072
:101EE000093C2B22A15CE26A12020A432721605CB2
:101EF000A16A090201432320255C606A000228438D
:101F0000E679257A2D023543039565790295257981
:101F100001952125645D0094FFF79CFAD5E71A4BE3
:101F20001C00093C2B22A15CE26A12020A43272111
:101F3000605CA16A090201432320255C606A0002FB
:101F40002843E679257A2D02354303956579029574
:101F5000257901952125645D0094FFF715F8B4E714
:101F60000A4804F0FBF97DE7938E0220AC8B022037
:101F7000B8950010C8950010AF8B0220408C02204D
:101F8000DC950010968E0220B58B0220EC95001097
:101F900030B585B003AB02AA01A9444800F0CAF8E5
:101FA000002803D14149424801F0D6FB039A029927
:101FB000019800F083F804F00FFAFA20800000F096
:101FC00027FF802200213B4804F062F8192000F02E
:101FD00021F9D0231B06802292045A6219E00134B1
:101FE000029B9C420DD2039B5A1C0392E85C04F0B6
:101FF00081F980239B02039A9A42F0D30023039332
:10200000EDE72D4B00221A70D0231B06802292048C
:102010009A61D0231B06802292045A61264B1B78BA
:10202000002B3FD0FFF72AFE00281FD102AC03A9E6
:102030002000FFF72BFE0500642000F0E9FE207869
:1020400004F058F9607804F055F9A07804F052F9DA
:10205000E07804F04FF9642000F0DAFE029B9B0068
:102060000293039B9B0003930024B9E7D0231B0634
:10207000802292049A61642000F0CAFE002004F0DD
:10208000AFF9431C05D0FEF75FFF0B4B00221A701F
:10209000BAE7D0231B06802292045A61642000F024
:1020A000B7FEB1E7FFF792FEAEE7C046400D030072
:1020B000FC950010AC8B0220968E0220F0B583B008
:1020C00004000D00160000F029F9002801D003B02B
:1020D000F0BD154F00973B0001220121053001F0B2
:1020E00053FB00962B0022000121104801F064FEF2
:1020F00031006943200003F071F804000C4B009399
:1021000000220221042001F03FFB00942300002262
:102110000121052001F038FB00973B00022200213D
:10212000062001F031FBD2E7006CDC0200800240A7
:10213000001BB700F0B5DE4657464E464546E0B5B3
:1021400083B080468B4600920193042001F01EFC70
:10215000FA21890003F042F88246A0235B009946E9
:102160002CE0013C002C20D025007D4329003000CC
:1021700003F034F84045F4D12900300003F02EF884
:102180000029EED173019B1B9B009E19F6005B4654
:102190001E60009B1F60019B1C60012003B0F0BC0F
:1021A000BB46B246A946A046F0BD013F002F01D074
:1021B0003C00D7E701235B429C46E1444B460F2B92
:1021C00009D956464B465E43044BF218044B9A42DB
:1021D000F0D80727EAE70020E0E7C04680E5F9FFEE
:1021E000804F120010B58300084A944663441C686F
:1021F00040226240C02414408022520113431C60DC
:10220000C000034B9C466044416010BD04C00140C7
:102210000040014010B501238340D0221206936292
:1022200093610521FFF7DEFF10BD0000EFF3108082
:1022300072B6034B1B68002BFBD0BFF35F8F704758
:102240002C0100D0BFF35F8F024B00221A6080F395
:10225000108870472C0100D0F8B506000C0015005E
:10226000FFF7E4FFE308F718F15C0722224001239F
:1022700093400B4205D1DBB20B433B70FFF7E2FF0B
:10228000F8BD2100280001F067FAF0B583B0060020
:10229000019114001F00FFF7C9FF00E00134BC42A8
:1022A0000CD8E308F518F35C0721214001228A408D
:1022B0001A42F3D1D2B21A432A7001E001246442D7
:1022C000FFF7C0FF002C02DB200003B0F0BD019B34
:1022D000002BF9D0089801F03FFA000070B5050016
:1022E0000C00FFF7A3FFE308EE18EA5C07210C409F
:1022F0000123A340134204D09A433270FFF7A2FF98
:1023000070BD034B034A2C31034801F08BF9C046E2
:10231000FC9600105C9700101C970010034B1B6884
:1023200002201840431E9841C0B2704700C00640CA
:10233000002307E0054A9A189200BFF35F8F00213F
:10234000116001331F2BF5D97047C046400000349F
:10235000054A1078431CDBB21370172B02D9130007
:1023600010221A707047C0464204002000B583B0A6
:102370000100044B00931F2318220348FFF785FF39
:1023800003B000BD6C970010D886022070B5050020
:102390000C00080000F0CCFD200000F0D5FE08493C
:1023A000200000F015FEFFF7D3FF064B9C4660446B
:1023B000800068602C75A400034BE55070BDC046DA
:1023C000D126001040000034308C02200A4B1A68DD
:1023D000EFF3108172B61368002BFCD0BFF35F8F50
:1023E000054B1B68BFF35F8F00221A6081F31088D2
:1023F00040BF002000217047508E022010B50029F8
:1024000022D003681B7B99421ED8174B9C4661441F
:10241000090183689C4661440C684968002A19D008
:1024200003681B7B9A4215D883680F488446624430
:1024300012019A1810685368020001208B4201D8DB
:102440000ED00020C0B210BD084B094A3B210948FC
:1024500001F0E8F8054B064A3B21064801F0E2F896
:10246000A242EFD8EDE7C046FFFFFF0FD497001060
:10247000909A00109C97001010B500291ED0037B85
:1024800099421BD84B005B18033B0468A446634485
:10249000002919D0002A1DD0914221D0002A25D030
:1024A000047BA24222D80468500080180338201808
:1024B0008170197800291FD11A7010BD104B114A74
:1024C0006821114801F0AEF8104B114A6F310E48E7
:1024D00001F0A8F80F4B0E4A70210B4801F0A2F84A
:1024E0000D4B0B4A7121084801F09CF8044B054A3A
:1024F0006821054801F096F841701A70DDE7C04682
:1025000008980010FC9A0010249800106C98001095
:10251000D89A0010789800108498001070B50600C2
:102520000D001400002914D0002A14D080687368AC
:102530009847002806D0220029003000FFF79CFFB2
:10254000280007E02A0021003000FFF795FF200057
:1025500000E0100070BD0800FCE70000F0B583B09B
:102560000500009201930AAB1C780BAB1F78002C7E
:1025700026D003685A7B944207D10123002B19D13E
:10258000002C3BD1200003B0F0BD002C0CD01A7BF6
:10259000944209D81A6863001B19033BD3189B782F
:1025A000002BEBD00123E9E73E4B3F4A68213F482F
:1025B00001F038F83E4B3F4A65213F4801F032F8C0
:1025C00003689C7B002CDBD012D01A7B94420FD87E
:1025D00062001219033A19688C4662445178997363
:1025E000002900D1D9730023937053701370C7E78B
:1025F0002C4B2D4A68212D4801F014F8002C3AD0BC
:102600002B681B7B9C4236D82C4BE3181B01AA6815
:1026100094466344009A1A60019A5A60089A9A6034
:10262000099ADA602E68002C2BD030D0337B9C4284
:102630002DD863001B19033B326894466344002283
:102640009A705A701A70717B22003000FFF766FF93
:102650007073844200D095E7287D009A019B00F0BA
:10266000FFFC061E01D0002F17D00C9B002B00D1C1
:1026700088E71E7086E7124B124A3B210E4800F095
:10268000D1FF114B114AA521084800F0CBFF054BA3
:10269000054A6821054800F0C5FF2868210000F0C0
:1026A0003FFFE2E708980010FC9A00102498001001
:1026B0009C980010089B00109C970010FFFFFF0FD4
:1026C000D4970010909A001098970010EC9A001080
:1026D000F0B5DE4657464E464546E0B58BB009900C
:1026E000002308938200B24BD658370032E0B14B3A
:1026F000B14A3F21B14800F095FFB14BB14A3B21AF
:10270000B14800F08FFFB14BB14A8C21AE4800F0C8
:1027100089FFB04BAE4A9021AB4800F083FFA84B35
:10272000AD4A4021A84800F07DFF2A686B680998EF
:1027300000F096FC00239A4698467B68BFF35F8FB3
:1027400000221A6086F310884346002B51D10028DE
:1027500000D126E100F0F8FB02000B1EC7DB0020D1
:102760000021069007917868EFF3108672B6016831
:102770000029FCD0BFF35F8F396888464C7B002C62
:1027800032D0BAD0097B8C42B7D8944965182D0154
:10279000B9688C46654428686968801A994100299F
:1027A000C3DC01D10028C0D10021404600F0AEFEBC
:1027B000A042A8D12A686B6806920793AB68984636
:1027C000EB689A464346002BA3D0002CA7D03B6869
:1027D0001B7B9C42A3D8631EFA68D35C08931B0240
:1027E000184338610020A8E700239A469846002045
:1027F000A3E7089B1B022343994651461800C04794
:1028000005000E007A68EFF3108B72B61368594218
:102810004B41D9B2002BF9D1BFF35F8F002E26DBDD
:10282000002E52DD3B69002B53D04B4572D100F096
:102830008BFB02000B1E73DB010018005219734161
:10284000984202D804D1914202D901225242D317B0
:10285000002B6BDB0021049101310391029451465E
:102860000191414600913800FFF778FE49E03B694D
:10287000002BD5D04B451CD1069A079B10001900A0
:10288000521BB341994202D804D1904202D901228D
:102890005242D317002B12DB002104910131039126
:1028A000029451460191414600913800FFF756FECF
:1028B00027E04B4B464A9F21434800F0B3FE3D4B77
:1028C0003D4A3F213D4800F0ADFE002E01D1002DD4
:1028D000A8D13A68002C45D0537B9C422CD10121D1
:1028E00000293FD1D37B002B42D1D473002C52D08E
:1028F0003B681B7B9C424ED8FA68013C135D013358
:10290000135500233B617A68BFF35F8F13608BF32D
:1029100010881FE7324B2E4AA2212B4800F082FE7E
:10292000244B254A3F21254800F07CFE214B224ABA
:102930003F21224800F076FE002C0DD0137B9C42F4
:102940000AD863001B19033B1068844663449B78D4
:10295000002BC5D00121C3E7224B234A682123481D
:1029600000F060FE224B234AF621204800F05AFE78
:10297000002B0AD0117B8B4207D85900CB18033BA0
:1029800011688C4663445C70AFE7164B164A6821A9
:10299000164800F047FE0A4B0F4A40210A4800F053
:1029A00041FE0BB0F0BCBB46B246A946A046F0BD06
:1029B000308C0220C49800105C9A0010E09800103F
:1029C000D4970010909A00109C9700102499001042
:1029D000749A00103C990010B49A0010FFFFFF0F8A
:1029E0004899001008980010FC9A001024980010D4
:1029F00084990010C89A001010B50A4B5B68002B30
:102A000004D00A21084800F0BFFB10BD054C23008C
:102A1000064A1021206800F099FC03212000FFF7EE
:102A2000B5FCEEE744040020508E0220FD23001088
:102A300010B5064B5B68002B01D0044810BD044B59
:102A4000044A5C21044800F0EDFDC0464404002027
:102A5000A89900109C9A00109C970010F0B5DE46D3
:102A600057464E464546E0B58BB0804616001F00DF
:102A7000149B9A46159B994616AB1B789B461F23C1
:102A800002AA9446634400221A7032E0002809D05A
:102A900042461268127B904204D8421E4146C968E1
:102AA0008A5C48E0434B444A4021444800F0BAFD68
:102AB0000798002B75D05B46002B72D04946D04753
:102AC00004000D0003000B4300D171E0002946DB38
:102AD00000F03AFA06000F1E55DB36196F41B94275
:102AE00002D804D1B04202D901267642F717002F4E
:102AF0004FDB43465A68EFF3108472B613685942AD
:102B00004B41D9B20791002BF8D1BFF35F8F1F3330
:102B100002AA9446634404930023039302934B4612
:102B200001935346009332003B004046FFF716FDE9
:102B3000031EABD1020041464968BFF35F8F0025F9
:102B40000D6084F31088002B29D01F2302A98C4626
:102B500063441B78002BABD112021043A9E732006B
:102B60003B00361BAF41BB4202D804D1B24202D96E
:102B700001267642F717002FBBDA114B114A3F218D
:102B8000114800F04FFD0E4B0E4A3F210E4800F059
:102B900049FD0B4B0B4A3F210B4800F043FD012040
:102BA00040420BB0F0BCBB46B246A946A046F0BDC1
:102BB0000798F6E7D4970010B49A00109C9700107D
:102BC000C49800105C9A0010E0980010F8B504005A
:102BD0004268EFF3108572B6136858424341D8B289
:102BE000002BF9D1BFF35F8FCBB22268567BB34283
:102BF0001BD10120002848D0206988422BD0090A27
:102C0000C9B2002B2ED02068007B83422AD8581EE0
:102C1000E668305C88422BD000206368BFF35F8F8A
:102C200000221A6085F31088F8BD002B0DD0167BAA
:102C3000B3420AD85E00F618033E1768BC466644E5
:102C4000B678002ED6D00120D4E7134B134A682162
:102C5000134800F0E7FC8521124B134A4900134842
:102C600000F0E0FC124B134A4021104800F0DAFC5F
:102C70001900100000F054FC0028CED112210E4B98
:102C8000094AFF31094800F0CDFC23698B42C4D1C9
:102C900000232361C1E7C04608980010FC9A001089
:102CA00024980010CC990010449A00109C970010B2
:102CB000D4970010B49A0010F0990010F0B587B0C6
:102CC00006000F00FDF7CFFA00281FD1062464424A
:102CD000E517A4197D41BD4202D803D1B44201D900
:102CE00000240025002D14DB0494059500F02CF938
:102CF00002000B1E13DBA41A9D41002D17DC14D01B
:102D00003000390000F02CF907B0F0BD234800F086
:102D100023FD234B234A3F21234800F083FC204B13
:102D2000204A3F21204800F07DFC002CE8D0FFF72E
:102D30007FFE0023029301931C4B0093049A059B92
:102D4000FFF78CFE002818DADAE7002300E0002302
:102D5000002BD5D1164B1A68EFF3108172B61368A9
:102D6000002BFCD0BFF35F8F114B1B68BFF35F8F4D
:102D700000221A6081F3108820BF0499059A0D4B38
:102D80005B6A9A42E3D80B48806A884203D29A422F
:102D9000DBD00123DCE70123DAE7C046F499001019
:102DA000C49800105C9A0010E0980010CD23001029
:102DB000508E022000400540F8B504000D0000F0E0
:102DC000C3F802000B1E10DB2000290080185941B7
:102DD0008B4202D804D1824202D901204042C1175D
:102DE000002908DBFFF76AFFF8BD064B064A3F21C2
:102DF000064800F017FC034B034A3F21034800F04C
:102E000011FCC046C49800105C9A0010E0980010B5
:102E100010B5FA2292000023002103F023F8FFF7F7
:102E2000CBFF10BD70B584B006000C00FFF700FEAC
:102E3000002302930193194B009332002300FFF704
:102E40000DFE051E11DD20BFFFF7F2FD2900FFF783
:102E5000BDFE134B5B6A9C421BD8114A926AB24278
:102E60001AD29C4213D0012014E00D4B5B6A9C42A5
:102E700009D80B4A926AB24207D29C4201D0012083
:102E800008E0002006E0002004E0012002E000202D
:102E900000E0002004B070BD0120FBE7CD2300104E
:102EA0000040054070B5EFF305833F20184010380F
:102EB000EFF3108C72B6194B1B68002BFBD0BFF3DD
:102EC0005F8F012319008140154A5163154A12781A
:102ED0001400C440234214D0114B5C6A8300124D8D
:102EE0005B599C4206D38300104C1B598A430D4901
:102EF0000A7007E00A4A031D9B0099589950002365
:102F000000E00023BFF35F8F044A002111608CF3BF
:102F10001088002B00D0984770BDC046280100D013
:102F200000400540A18E0220648E0220C085022050
:102F300010B50100024A0348FFF78EF910BDC046E4
:102F4000209B0010978E0220044B5B6A034A906A14
:102F50001900536A9942F9D17047C04600400540B4
:102F6000084B5B6A01E0074B5B6A8B42FBD301E0D5
:102F7000044B5B6A8B4203D1024B9B6A8342F7D3BB
:102F80007047C0460040054070B504000D00FFF7D3
:102F9000DBFF02000B0020002900801859418B4202
:102FA00002D804D1824202D901204042C11700292F
:102FB00002DBFFF7D5FF70BD024B034A3F210348F8
:102FC00000F030FBC4980010C49B0010E098001083
:102FD00070B504000D00EFF3108672B61B4B1B6832
:102FE000002BFBD0BFF35F8F002D1CD0200000F022
:102FF00057FD174B83420BD01900200000F058FDFD
:103000000121200000F03CFD0123A340114A136080
:10301000A400114BE550BFF35F8F0C4B00221A60E8
:1030200086F3108870BDA2000B4B0021D150012205
:10303000A2400A490B7893430B700549200000F029
:1030400061FD0021200000F01BFDE4E7280100D015
:10305000A52E001038600540C0850220A18E0220F8
:10306000F0B5DE4600B584B00400150001921E00E4
:103070000293FFF769FF03958E4202D84ED1854235
:103080004CD9EFF3108B72B6274B1B68002BFBD08B
:10309000BFF35F8F254A17780125A540EBB23B436C
:1030A0001370234B5D63221D92000199D150A20041
:1030B0002049029850501B6A2B4212D11C4B1B6CAA
:1030C0002B4208D00020BFF35F8F174B00221A60FD
:1030D0008BF3108823E0184B184AC121184800F0E0
:1030E000A1FAFFF731FF8E4214D802D1039B83422D
:1030F00010D80E4B1B78BB420ED00D4B1D625D638A
:103100001F2004400123A3400E4A1360074B1F7089
:103110001E38D8E70020D6E70120D4E7012004B00C
:1031200080BCBB46F0BDC046280100D0A18E022065
:1031300000400540648E0220449B0010A89B0010B4
:10314000689B001080E200E0EFF3108C72B60B4B2E
:103150001B68002BFBD0BFF35F8F01238340084A1D
:10316000136208490A789A430A70BFF35F8F034BD2
:1031700000221A608CF310887047C046280100D0E6
:1031800000400540A18E0220024B9C46614489000C
:10319000016070474000003410B50400FFF7D8F814
:1031A00001002000FFF7F0FFFF232371BFF35F8FC3
:1031B00010BD10B50400FFF7CBF801002000FFF7A9
:1031C000E3FFFF23237100236371BFF35F8F10BD03
:1031D000034B9C46614489000160BFF35F8F7047D9
:1031E0004000003410B504000120FFF7BFF80100D3
:1031F0002000FFF7EDFF10BD10B500291ED0037BA6
:1032000099421BD84B005B18033B0468A4466344F7
:10321000002919D0002A1DD0914221D0002A25D0A2
:10322000047BA24222D8046850008018033820187A
:103230008170197800291FD11A7010BD104B114AE6
:103240006821114800F0EEF9104B114A6F310E4819
:1032500000F0E8F90F4B0E4A70210B4800F0E2F93C
:103260000D4B0B4A7121084800F0DCF9044B054A6C
:103270006821054800F0D6F941701A70DDE7C046B4
:1032800008980010989D0010249800106C98001069
:10329000849D0010789800108498001070B5060086
:1032A0000D001400002914D0002A14D0806873681F
:1032B0009847002806D0220029003000FFF79CFF25
:1032C000280007E02A0021003000FFF795FF2000CA
:1032D00000E0100070BD0800FCE7000010B50023FE
:1032E000437301338373037BC3730123027B9A42CD
:1032F00014D9002B0CD0027B934209D85A00D21863
:10330000033A01688C4662440133DBB25370EDE747
:103310000B4B0C4A68210C4800F084F9002A09D0B4
:10332000924207D8016853009A18033A8A1800237A
:10333000537010BD024B034A6821034800F072F934
:1033400008980010989D00102498001010B5017383
:1033500042608360FFF7C2FF10BD000070B504003B
:10336000081E00D170BD002934D0237B994231D88A
:103370004B005B18033B2268944663445A78002A4A
:10338000F0D02DD0237B9A422AD853009B18033BC0
:1033900021688C4663445D7800215970002825D04F
:1033A000237B984222D843001B18033B21688C469C
:1033B00063440021597001002000FFF76FFF0600F1
:1033C00029002000FFF7CAFF020031002000FFF7AC
:1033D00065FFC7E7084B094A6821094800F022F950
:1033E000054B064A6821064800F01CF9024B034AC7
:1033F0006821034800F016F908980010989D001005
:103400002498001070B505000C001600002928D083
:103410002DD0037B99422AD84B005B18033B0268EE
:10342000944663445A78002A27D19A78002A2AD1F0
:103430001978FFF793FF0300002E03D0EA7B002AE0
:1034400027D1EC73002B37D1002C49D02B7B9C4229
:1034500046D82B6861000C19033C1C1900236370CB
:1034600070BD224B224A3821224800F0DBF8224B63
:10347000224A6821224800F0D5F8224B1C4A3A2102
:103480001C4800F0CFF8204B194A3B21194800F0A6
:10349000C9F8002A0AD0297B8A4207D851008A1825
:1034A000033A29688C4662445470CAE7124B134AA7
:1034B0006821134800F0B6F8002B0BD02A7B93420A
:1034C00008D843001B18033B2A6894466344002233
:1034D0009A70B9E7084B094A6821094800F0A2F838
:1034E000054B064A6821064800F09CF8A49C001091
:1034F000709D0010AC9C001008980010989D001062
:1035000024980010E49C00100C9D001070B504007D
:103510000A00457B2900FFF775FF6073280070BD26
:1035200070B50400002967D0437B8B420ED0002980
:1035300011D0037B99420ED84B005B18033B026805
:10354000D0188378002B0CD1002056E00121FFF722
:10355000DDFF012051E0294B294A6821294800F06C
:1035600061F8002B20D0227B93421DD85A00D3183B
:10357000033B2268D2182568EB5C8B421AD0002BE3
:103580001BD0227B934218D85A00D318033B2268E1
:10359000D21853788B4216D0002BF0D11A4B1B4A0D
:1035A00067211B4800F03EF8144B154A6821154866
:1035B00000F038F84378137007E0104B104A682188
:1035C000104800F02FF84378537000238370437045
:1035D00001222000FFF716FF0200617B814205D027
:1035E0002000FFF75BFE6073012006E0094B074AED
:1035F0006D21074800F016F8002070BD08980010F3
:10360000989D001024980010309D0010589D0010C7
:10361000AC9C0010389D001000BEFDE710B5FFF710
:10362000FBFF000010B582B00C001900002A0CD07E
:10363000084B002A0BD00192009323000200064899
:1036400002F0BEFE0120FFF7E7FF044BF1E7034A5B
:10365000F1E7C046A49D0010B49D0010B09D00107D
:1036600070B52B4B2B4A1A602B4B2C4A1A602C4BF3
:103670009A682A4B9343FAD12A4C01E008CC984728
:10368000294B9C42FAD300F001F9234B274A1A60D8
:10369000234B9B68DB43DB01FAD1254B40229A6721
:1036A0005A671A67DA66234C09E0234B234A8321C1
:1036B0002348FFF7B7FF2000FFF76EFD0834214BCA
:1036C0009C4209D22368002BF5D0012BEDD12000BC
:1036D000FFF76FFD0834F2E71B4CA1681B4DC022B9
:1036E000280002F0DBFCA560FCF7BDFD002800D03F
:1036F00000BEFEF71DFE00F051FBFFF77DF9144CF4
:1037000001E008CC9847134B9C42FAD370BDC046E9
:1037100000E00040BFCDFBFE00F00040FE7F3C001B
:1037200000C000403005002040050020FFFFFF01E1
:1037300000F0014020050020E49D0010589E00107C
:10374000049E00103005002000ED00E00000002085
:1037500040050020480500200FB400B583B008489C
:1037600002F0FCFD049B002B07D005A90191180075
:1037700002F004FE034802F0F1FD0120FFF74CFFC8
:10378000449E0010549E0010F8B5DE4657464E4643
:103790004546E0B505000F0092460A9A93424ED383
:1037A0001A0E91461E020A9A00233000494601F083
:1037B00057FD80466C006419A4002F4B9C4664445E
:1037C0006368834200D260602B1FDBB29B46012BF3
:1037D0003BD9C0239B012343802212011A60AB0016
:1037E000264A9958002905D0506901F0F7FC0130AC
:1037F0000138FDD153465A0123685A40E0231A404C
:1038000080235B0123431A605A46012A28D980236A
:103810009B012343802212011A60434663604246A3
:1038200000233000494601F01BFDAD00134B5851F9
:103830000120F0BCBB46B246A946A046F8BD104BDD
:10384000104A2D211048FFF7EDFE012FC1D1C023F2
:103850009B01234303221A60A368DB07FCD5C9E759
:103860002168794003220A401A60A2680123BB4004
:103870001342FAD0CBE7C04600800040DC8602202D
:10388000689E0010C09E00107C9E001030B583B072
:103890000C2000F021FBFEF741FD00280DD0002395
:1038A00004E099002D4A2E4888500133092BF8D99D
:1038B0002A4B2C4A5A6203B030BD2B4B00229A6728
:1038C00000F07CFB294B01221A60274B5B6C012B1B
:1038D000FBD1274B03221A60234B9B6B012BFBD19F
:1038E000022400940533234A0121234800F064FA9E
:1038F00000940523214A0121214800F05DFA214B63
:103900000093002202210420FFF73EFF1E4D009588
:103910002B00002201210520FFF736FF104C0094F8
:103920002300002200210720FFF72EFF0094230030
:10393000002200210820FFF727FF0A4B00932300F5
:10394000002200210920FFF71FFF00952B00002215
:1039500000210620FFF718FFADE7C046DC860220F5
:10396000006CDC021BB70000008000403CB000404F
:1039700030B00040002F68590080024000389C1C85
:1039800000C00240001BB700405973078000014B84
:10399000C0587047DC860220074B9B6810308000BF
:1039A0001950BFF35F8FBFF35F8F044B0021196085
:1039B00082F310887047C04600ED00E0240100D07B
:1039C00010B5091A081F0A4B9C466144094A9142E6
:1039D00008D8C30706D440104005400D064B1843D5
:1039E00080B210BD054B064A8B210648FFF71AFE30
:1039F000FC070000FE0F000000E0FFFFD09E00105B
:103A000008A10010009F001010B5091A04394C08D5
:103A1000090B08D14905490D064A11430180064B9F
:103A20002343438010BD054B054A93210548FFF70A
:103A3000F9FDC04600F0FFFF00F8FFFF3C9F0010BB
:103A4000DCA00010009F001001238340034A10688F
:103A50001840431E9841C0B27047C04600E100E0E4
:103A6000002904D0034B1860034B18607047034BC8
:103A70001860FBE780E200E000E100E080E100E0A8
:103A800010B5012383401800FFF7EAFF10BD0000C6
:103A900001238340014A13607047C04600E200E002
:103AA000024B9B6810308000C058704700ED00E06A
:103AB00070B504000D00EFF3108672B60C4B1B6856
:103AC000002BFBD0BFF35F8F2000FFF7E9FF094B0E
:103AD000984201D0A84205D1320029002000FFF70A
:103AE0005BFF70BD044B054A6E210548FFF79AFD48
:103AF000240100D0CD0100104C9F001024A1001023
:103B0000009F0010F0B5CE46474680B583B0060052
:103B10000D00EFF3108872B6564B1B68002BFBD0DC
:103B2000BFF35F8F544B9A6834001034A300D7580A
:103B3000524B9F4207D0AF4200D199E00197504BC2
:103B4000FB1A2F2B09D9424639003000FFF724FF1A
:103B500003B0C0BCB946B046F0BD3000FFF774FFFB
:103B6000814600213000FFF78BFFBFF35F8FFCF72A
:103B70007AFB002801D0844211D10123019C9C438F
:103B80000022A368AB4212D00622A256002A0DDB07
:103B900053009B189B002200394CE418F1E71E21CA
:103BA000384B394AFF313948FFF73CFD2200AB4220
:103BB00057D106256557002D39DB6B005B199A003C
:103BC0002F4B9B189A68A260DA79E27106229A5606
:103BD000A2719B795BB2002B10DABD200002A0809D
:103BE0006B005B199B00264AD318294A11789971FA
:103BF000157049463000FFF743FFA4E7201D6B0016
:103C00005B199B001E4A9B181A1D9B88D90A1C2908
:103C100007D15B055B15023359005118FFF7D0FE41
:103C2000DDE71C4B1C4A99211848FFF7FBFC0028D4
:103C300012D1002A0ED0FF239371184B9380144A9F
:103C40001378A371164B0E49641A644163431B0D2C
:103C50001370CEE7094FF2E7201D1249FFF7D4FE9B
:103C6000C7E75221104B084AFF310848FFF7DAFC3A
:103C7000024F68E7240100D000ED00E0CD01001004
:103C80006C04002060A00010F4A00010009F001041
:103C9000998E022048A0001014A1001000BDFFFF63
:103CA000AAAA0000A604002084A0001070B5040099
:103CB000012606432D4BF31A2F2B28D8FCF7D3FAF5
:103CC00000282BD0EFF3108C72B6294B1B68002B09
:103CD000FBD0BFF35F8F274D22002449521A524177
:103CE00055432D0D6DB2244B9B6880001B58B34289
:103CF0001BD00022032A32D853009B189B001B497B
:103D0000CB189B795BB2AB421FD00132F2E7BB21EB
:103D10001A4B1B4A49001B48FFF784FC7A211A4BB7
:103D2000174AFF311748FFF77DFC134B9B68174A72
:103D30001A50174B1A78A2711D70BFF35F8F0C4B8E
:103D400000221A608CF3108870BD08005300991887
:103D500089004118FF268E710E4A8A80E9E7C52145
:103D60000D4B074A49000748FFF75CFC6C04002034
:103D7000240100D0AAAA000000ED00E08CA00010F1
:103D8000C0A00010009F0010B4A00010CD010010D2
:103D9000998E022000BDFFFF309D00100022044BD1
:103DA00002E0044902C30132072AFAD97047C0462B
:103DB00000E400E080808080F0B5CE4600B50400CD
:103DC0000F0091461D000C2001F008FA0600430187
:103DD0001B1A9901C91AC90009188901484601F03E
:103DE000FDF90200103A98235B009A4233D86B1E0B
:103DF000062B36D8069B013B062B32D8069B9D42EC
:103E000035D34B461A09B24237D32D04069B1E0305
:103E100035432368002B36DB254B9C4244D080225F
:103E20005201244B1A60244B1A60244B9B681100EA
:103E30009943FAD12760A060231DC02292011A4342
:103E4000212313602368002BFCDAE560082313604C
:103E500080BCB946F0BD1A4B1A4A16211A48FFF722
:103E6000E1FB1A4B174A19211748FFF7DBFB184BE8
:103E7000144A1F211448FFF7D5FB164B114A222183
:103E80001148FFF7CFFB22683F231340BB42C3D149
:103E9000A3681B051B0D8342BED1E368EE22D2024C
:103EA0001340AB42B8D1D3E780229201B9E7C046B4
:103EB00000C0024000E0004000F0004000C00040B0
:103EC00040A1001018A200105CA1001098A10010E1
:103ED000E4A10010FCA1001080239B000343014AD1
:103EE000D362704700800540024B1A68024B5A604B
:103EF0007047C046A88B02200080054010B5020024
:103F0000164B8020C0051860154B16481860002914
:103F10000AD0154BE021C9041960002A09D1124BBF
:103F2000802212061A6010BD0C4BE021C9041960F2
:103F3000F3E753019B1A9800801800010B4B18609F
:103F400080235B04984202D3084B094A1A60FFF7AA
:103F5000CBFF054B8022D2051A60E4E700B0054094
:103F600008200140FCFF010000A00540A88B0220B2
:103F7000FFFFFF0010B5030010000C4A8024E40589
:103F80001460002B0DD001221343094A094CD4615F
:103F9000094C5C401462516293620021FFF7AEFF4E
:103FA00010BD034B0022DA61F7E7C04600B00540C0
:103FB00000800540D3C007B02D3FF84F064BAA2222
:103FC00012011A602F22DA60044B054A1A60024B74
:103FD0005B68002BFBDA7047004002400060024043
:103FE00000B0FA00704710B5002802D00B6849688D
:103FF000984710BD0100002007E083001B185B00FC
:10400000501C08601078C01830380A681378303BAC
:10401000DBB2092BF1D97047F0B5DE4657464E4664
:104020004546E0B583B093461F000C9B9A460D9C15
:104030000E9B99460F9B9B0703D0B8460F000600C6
:1040400022E00192A34688464E46B9460700B44294
:1040500007D2551C4B4641462020B84701342A0060
:10406000F5E73D004F465C46019B9B46B146464600
:10407000B84637002E0007E0013C551C5346185D3A
:1040800043463900B0472A00002CF5D135003E00E8
:1040900047460F9B9B0707D4100003B0F0BCBB46FC
:1040A000B246A946A046F0BDB0464E46B9462F00DE
:1040B0005D46531BB342EFD2541C4B464146202071
:1040C000B8472200F5E7F0B5CE46474680B585B043
:1040D000944698460C9D0D9C0EAB1B789946109A01
:1040E000119B129EB7071CD4002B0CD0F7070AD5E2
:1040F0004F46002F02D10C37374204D0013B02E07B
:1041000030272F550134944201D21F2CF8D9F707DC
:1041100007D59C4205D21F2C03D830272F550134D8
:10412000F5E7F70615D5770505D4002C03D09442A2
:1041300024D09C4222D00F9A102A2BD00F9A102AFA
:1041400030D00F9A022A35D01F2C02D830222A559F
:1041500001341F2C05D84A46002A31D02D222A5579
:104160000134039602930194009543466246FFF79B
:1041700053FF05B0C0BCB946B046F0BD621E012C6D
:1041800006D00F9F102F01D01400D4E7023CD2E7D5
:104190001400D0E7B206D1D41F2CCFD878222A55EC
:1041A0000134D1E7B206CCD51F2CCAD858222A55E3
:1041B0000134C9E71F2CC7D860322A550134C3E740
:1041C000720703D52B222A550134CAE73207C8D516
:1041D00020222A550134C4E7F0B5DE4657464E4644
:1041E0004546E0B593B081468A46089209931CABD8
:1041F00010CB1B789B461E9D219B9846002C03D11B
:10420000102342469A4390468023DB0046461E40D8
:1042100042461A4212D0002C22D000260EE0303343
:10422000D9B2771C0AAB99552900200000F0D6FFBF
:10423000AC4216D31F2F14D83E00040029002000E2
:1042400000F0CCFFCBB2092BE9D94246920605D546
:104250004121C918C9B20A39C9B2E2E76121F8E7B8
:10426000270043460693209B05931F9B04930395C9
:104270005B46029301970AAB0093099B089A51464B
:104280004846FFF720FF13B0F0BCBB46B246A94634
:10429000A046F0BDF0B5DE4657464E464546E0B571
:1042A00095B0089009910A920B931E9E1F9C20AB1B
:1042B0001B789B46229B9946239D269B9A4633005A
:1042C000234303D1103352469A4392468023DB00A6
:1042D00057461F4052461A4219D0330023432DD06F
:1042E000002714E03033DAB27B1C98460CABDA5569
:1042F0004A462B003000210000F0B2FFA5421FD833
:1043000019D043461F2B1BD8474606000C004A46CF
:104310002B003000210000F0A3FFD3B2092BE1D91C
:104320005246920605D54122D218D2B20A3AD2B2EA
:10433000DAE76122F8E7B145E3D901E000239846C6
:1043400053460693259B0593249B04934B46039366
:104350005B460293434601930CAB00930B9B0A9A76
:1043600009990898FFF7AFFE15B0F0BCBB46B246FE
:10437000A946A046F0BD0000F0B5DE4657464E46C1
:104380004546E0B591B083468A460C9298461A9C01
:1043900008941B9D099522002B002000290001F0A4
:1043A000EEF9002800D0E5E001225242D74B200070
:1043B000290001F0DFF9002800D0DBE001225242A1
:1043C000D34B2000290001F0BFF9002800D0D1E034
:1043D00000220023089E3000099D290001F0B4F955
:1043E000002800D0DDE00898099906900791802305
:1043F000DB001E9A1A400D921E9A1A4201D1062322
:104400001C930698079904000D000A000600024359
:1044100000D1D1E0080D4005400DBE4CA4466044DB
:104420000A03120BBC4B13431F0001F0BBF9BB4A3C
:10443000BB4B01F046F9BB4ABB4B01F01BF9040032
:104440000D000022B94B3000390001F00AF9B84ADA
:10445000B84B01F036F902000B002000290001F0F2
:1044600009F901F0B7F9814601F09CF904000D004B
:10447000B14AB24B01F025F90022B14B01F0FAF834
:1044800001F0A8F90600AF4AAF4B2000290001F067
:1044900018F904000D00300001F084F9AB4AAC4B70
:1044A00001F00FF902000B002000290001F0D9F8FB
:1044B00004000D0002000B0001F003F90A900B91BB
:1044C000A44BF31800261F0522002B002000290012
:1044D00001F0D0F80E900F9122002B0000208021D7
:1044E000C90501F0BEF804000D0000229A4B0A989D
:1044F0000B9901F0C8F80022984B01F0BBF80200BC
:104500000B000A980B9901F0BEF80022944B01F0C1
:10451000B1F802000B000A980B9901F0B4F8020000
:104520000B002000290001F0A5F802000B000E98F6
:104530000F9901F0A8F80022774B01F09BF83200A8
:104540003B0001F0BEF806000F0004000D00069AC3
:10455000079B01F00FF9002830D001235B429C46F5
:10456000E14400227D4B3000390001F08CF804005A
:104570000D0023E01E9B04931D9B03931C9B029341
:10458000089A099B0092019343460C9A514658465B
:1045900000F0FCF811B0F0BCBB46B246A946A046FC
:1045A000F0BD0023002406930794069680231B0683
:1045B0009C46654407951AE7002399464B466333AA
:1045C000C62B1ED804261E9B1B0526D52B00234375
:1045D0000FD0644A644B0698079901F0C3F800288D
:1045E00079D00022614B0698079901F0ADF80028B8
:1045F00071D01C9B4B4506DD4A46981A431E1C93FE
:1046000003E00526DFE700231C938023DB001E9ACE
:104610001A431E920026002399461D9B9E4264D297
:104620009F1B02231E9A1A400A921E9A134202D01E
:10463000002E00D000274B46002B07D022002B0075
:104640000698079901F01FF80690079100220023B1
:104650000898099901F078F8002848D1444B1E9A2F
:104660001340049303971C9B0293069B079C0093A3
:10467000019443460C9A5146584600F087F8002EA4
:1046800000D187E71E9B9B063DD54525441C43462C
:10469000020051462800D8474B46DA179B18534072
:1046A00005220592013E0496002203920A320292EC
:1046B0004A46D00F01900093434622005146584687
:1046C000FFF78AFD0A9B002B00D163E702005F46DB
:1046D0000C9E1D9D54E01C9B002B9ED00D9B002B1F
:1046E0009BD01C9B013B1C9397E7002799E7069CF6
:1046F000079D2200290080200006844661440B00AB
:1047000006920793AAE76525C0E7C046FFFFEF7F43
:10471000FFFFEFFF01FCFFFF0000F03FFB799F5020
:104720001344D33FB3C8608B288AC63F0000F83FCC
:1047300061436F63A787D23F71A379094F930A4002
:104740000000E03F1655B5BBB16B0240EF39FAFEF1
:10475000422EE63FFF03000000002C4000002440F2
:10476000000018402D431CEBE2361A3F80842E4196
:10477000FFF7FFFF541C434651462020B847220054
:10478000931BAB42F6D3100004E7C046F0B5DE46FB
:1047900057464E464546E0B595B00690079193467C
:1047A0009946209F1E9A1F9B1000190000F0E7FFFA
:1047B000002831D101225242BF4B1E981F9900F0B0
:1047C000C3FF002837D101225242BC4B1E981F99CB
:1047D00000F0D0FF00283DD10022B94B1E981F9950
:1047E00000F0C8FF002850D10022B64B1E981F9938
:1047F00000F0AAFF002848D1002200231E981F992C
:1048000000F0A2FF002850D100239846229B5B05B0
:1048100000D4B6E0002458E0229B0393219B02932E
:1048200003230193A84B00934B465A4607990698D9
:10483000FFF7F2FB0EE1229B0393219B02930423DB
:104840000193A24B00934B465A4607990698FFF7EF
:10485000E3FBFFE00423229A1A4022990B4210D076
:104860009B4B002A0FD00422229903912199029197
:10487000019200934B465A4607990698FFF7CCFBE6
:10488000E8E0944BEDE70322EEE7229B0493219BA3
:10489000039302971E9B1F9C009301944B465A461C
:1048A00007990698FFF768FDD4E01E9A1F9B002029
:1048B000002100F0D6FE1E901F9101239846A5E727
:1048C0000CAB30221A55013F01341F2C01D8092F9F
:1048D000F6D81E981F9900F07DFF050000F062FFDA
:1048E00002000B001E981F9900F0BBFEFA007A4BE5
:1048F0009B181A685B680A920B9300F0E2FE08901E
:10490000099100F08BFF060000F048FF02000B0049
:104910000898099900F0A5FE0890099100226F4BB4
:1049200000F028FF00282ED00136300000F036FFBE
:1049300002000B000A980B9900F00CFF002801D030
:1049400001350026002F2CD1280000F02BFF02009B
:104950000B001E981F9900F084FE06000F00002235
:104960005E4B00F0F1FE002846D100225B4B300088
:10497000390000F0FFFE00283ED1EB073CD50135A1
:104980003AE0062746E70022544B0898099900F0C0
:10499000DBFE0028D6D1002E01D0F307D2D5013698
:1049A000D0E7AA461F2C11D8013F0A21300000F0A1
:1049B00015FC651C30310CAB19550A21300000F094
:1049C0000DFC092E0ED906002C00EBE755461F2CD6
:1049D0000CD87B1E002F09D00CAA302111551F00C6
:1049E0000134F4E72B0055461C00F0E71F2C03D8D8
:1049F0000CAB2E221A5501341F2C10D80A21280086
:104A000000F0C4FB661C30310CAB19550A2128009C
:104A100000F0BCFB051E01D03400EDE73400032399
:104A2000229A1340012B1CD01F2C06D84346002B82
:104A300032D00CAB2D221A550134229B0393219BBB
:104A4000029301940CAB00934B465A460799069883
:104A5000FFF7E2FA15B0F0BCBB46B246A946A04645
:104A6000F0BD219B002B13D04346002B02D10C3309
:104A700013420FD0219B013B2193190003E00CABA3
:104A800030221A5501348C42CED21F2CF7D9CBE7F5
:104A90002199F8E72199F6E7229B5B0704D50CAB37
:104AA0002B221A550134C8E7229B1B07C5D50CAB36
:104AB00020221A550134C0E7FFFFEFFFFFFFEF7F11
:104AC00065CDCD4165CDCDC130A2001034A200101E
:104AD00028A2001024A2001020A400100000E03F33
:104AE000F0B5DE4657464E464546E0B593B08246A1
:104AF0008B4690461193002900D1EBE200275546E2
:104B0000119B1878002800D1E7E2252809D07C1CE9
:104B100043463A005946A847119B01331193270099
:104B2000EEE7013311930024119A11780B00203B1A
:104B3000D8B2102803D88300D048C3589F460B0032
:104B4000303BDBB2092B2CD92A292FD000230A9322
:104B5000119B1A782E2A39D000239A46119A13787D
:104B6000683BD9B2122976D88B00C549CB589F46ED
:104B700001231C4301321192D6E702231C43013268
:104B80001192D1E704231C4301321192CCE7082390
:104B90001C4301321192C7E710231C4301321192CA
:104BA000C2E711A8FFF726FA0A90D1E71C9B1A1D4D
:104BB0001C921868002804DB0A90119B01331193A2
:104BC000C6E702231C4343420A93F6E78022D20041
:104BD00014435A1C11925A781300303BDBB2092B54
:104BE00004D92A2A07D000239A46B7E711A8FFF76D
:104BF00001FA8246B2E71C9B1A1D1C921868002815
:104C000004DB8246119B01331193A7E70020F8E7EC
:104C100080235B002343511C119152786C2A01D0F0
:104C20001C0018E0C0239B001C430131119112E0CD
:104C300080232343511C11915278682A01D01C0013
:104C400009E0C0231C430131119104E080235B0083
:104C50001C4301321192119B18780300253BDAB2F4
:104C6000532A00D92CE29300864AD3589F468023CA
:104C70009B001C4301321192EDE780235B001C4333
:104C800001321192E7E7782809D0582838D06F28E8
:104C900038D0622838D010239C430A2600E0102622
:104CA000582833D0692803D0642801D00C229443BB
:104CB000630501D50122944369282AD0642828D0AD
:104CC000A30500D59FE0E30500D5B8E0630600D456
:104CD000CAE01C9A111D1C911168FF220A4005941C
:104CE0000A9B049353460393029600230193009278
:104CF00043463A0059462800FFF76EFA070027E0BE
:104D00001026CDE70826CBE70226C9E72022144368
:104D1000C8E7A30520D4E30550D4630666D51C9AE2
:104D2000111D1C911168FF220A40D317D118594058
:104D300005940A9B0493534603930296D20F019263
:104D4000009143463A0059462800FFF745FA07000C
:104D5000119B01331193D3E61C9BDA1D07218A4373
:104D6000110008311C91116853689C46DB170C93A5
:104D70000D930C9A0D9B100048400E9062465340D4
:104D80000F930E980F990C9A0D9B801A99410E90D3
:104D90000F9108940A9B07935346069304960023A9
:104DA00005936346DA0F02920090019143463A0060
:104DB00059462800FFF76EFA0700C9E71C9A111D33
:104DC0001C911268D317D118594005940A9B04937B
:104DD000534603930296D20F0192009143463A0044
:104DE00059462800FFF7F8F90700B1E7230605D573
:104DF0001C9A111D1C910023D25E96E71C9A111D6E
:104E00001C91126891E71C9BDA1D07218A4311004F
:104E100008311C9108940A9B079353460693049605
:104E2000002305930293136854680093019443464A
:104E30003A0059462800FFF72DFA070088E71C9A28
:104E4000111D1C9105940A9B0493534603930296EB
:104E5000002301931368009343463A005946280003
:104E6000FFF7BAF9070073E723060DD51C9A111D49
:104E70001C9112681204120C31E7C0463CA20010CB
:104E800080A20010CCA200101C9A111D1C91126867
:104E900025E746281AD01C9B0733072293431A00A4
:104EA00008321C9204940A9A0392524602925C6859
:104EB0001B680093019443463A0059462800FFF7C7
:104EC00065FC0700119B0133119319E620231C4355
:104ED000E1E7672801D0472802D180231B011C434A
:104EE000452801D0472801D120231C431C9B0733B0
:104EF000072293431A0008321C9204940A9A0392E0
:104F0000524602925C681B680093019443463A0043
:104F100059462800FFF730FA0700119B013311931F
:104F2000EEE502231A002240924623421FD00124BC
:104F30001C9B1A1D1C927A1C9146187843463A0015
:104F40005946A8475346002B16D1119B01331193A4
:104F50004F46D5E5561C434659462020B847230006
:104F600032005C1C9D42F5D83D001700E0E70123AC
:104F70003A002F000A9DF4E74A46A9460A9D06E03A
:104F8000571C434659462020C84734003A00661C47
:104F9000A542F5D84D469146D7E71C9B1A1D1C9299
:104FA0001B6899465346002B00D1013B4E4601E059
:104FB000013613003278002A02D05A1E002BF7D196
:104FC0004B46F21A10928023DB0026001E401C4242
:104FD00003D0524501D95346109302231A002240B0
:104FE0000B92234205D03A0037004C46A94655465D
:104FF00020E03A00109B5F46B3462E0006E0551CA9
:10500000434639002020B04723002A005C1C0A993F
:105010009942F4D835005E46BB46109437004C46A2
:10502000A946554606E01D000134561C4346594624
:10503000C84732002078002804D0002FF4D06B1E1F
:10504000002DF0D117004D460B9B002B03D1119B77
:105050000133119354E50A9F109B06E0561C43460A
:1050600059462020A847230032005C1C9F42F5D8F7
:105070001700ECE721231C431C9B1A1D1C921B6884
:10508000009305940823049353460393102302933B
:105090000023019343463A0059462800FFF79CF845
:1050A0000700119B013311932AE57C1C43463A000B
:1050B00059462520A847119B0133119327001FE56E
:1050C0007C1C43463A005946A847119B0133119373
:1050D000270015E50A4B9A4610E5AA46474502D334
:1050E00043465A1E00E03A00434659460020D04746
:1050F000380013B0F0BCBB46B246A946A046F0BD8E
:10510000E53F001000B585B00290039101210093A6
:1051100013004A4202A90248FFF7E2FC05B000BDB5
:10512000E73F001001480421014B1847C00400204C
:105130005551001010B5010018231B881422108847
:10514000984710BD10B5010018231B88162210883F
:10515000984710BDF0B5C64600B507000E00002503
:105160000123984600E00135B5420AD2AC003C1953
:105170002068FFF7DFFF20600028F4D10023984665
:10518000F1E7404680BCB846F0BD0000124A936F7C
:105190009B0815D29066D166002905D0FFE7FFE78E
:1051A000FFE7516F106F704704B580210906C217E1
:1051B0005140002800D0C84304F09EF9002104BDEE
:1051C000F0B5146E556E576F166FFFF7E3FF146658
:1051D000556657671667F0BD000000D0114A936FFF
:1051E0009B0813D210665166002905D0FFE7FFE740
:1051F000FFE7516F106F704704B5002801D0002001
:10520000C04304F079F9002104BDC046F0B5146E26
:10521000556E576F166FFFF7E5FF146655665767B3
:105220001667F0BD000000D094464E4A926F920877
:10523000624601D230E0C046F0B54A4EB56F6D0807
:10524000FCD3346E756E776F366F00F025F8944698
:10525000444A14665566576716676246F0BDC046F5
:105260009446404A926F9208624601D258E0C04686
:10527000F0B53C4EB56F6D08FCD3346E756E776F2C
:10528000366F00F04DF89446364A146655665767F7
:1052900016676246F0BDC046002B24DB11D0002902
:1052A0003EDA00B5C943404200D1013100F038F880
:1052B000C943404200D10131DB43524200D10133A6
:1052C00000BD002AEBD1002801D1002905D0002023
:1052D000C90FC90701D1C043410800B504F004F962
:1052E0000022002300BD00B500290ADBDB43524247
:1052F00000D1013300F014F8C943404200D101311C
:1053000000BDC943404200D10131DB43524200D1CC
:10531000013300F005F8DB43524200D1013300BDF8
:10532000002923D1002B18D1002A0CD0BC460D4FE8
:1053300038667A6600210023FFE7FFE7FFE77A6F10
:10534000386F67467047002801D00748010000B554
:1053500004F0CAF80022002300BD02000B00002068
:1053600000217047000000D0FFFFFFFF002B00D09E
:10537000BFE0130C28D1002AE7D080B4114F396662
:105380007A66FFE7FFE730B4040C7B6F396F1B04CC
:1053900023433B667A66FFE7FFE7FFE7C04684B238
:1053A0007B6F3D6F1B0423433B667A66FFE7FFE795
:1053B000C04600232C042D0C7A6F386F0019694108
:1053C000B0BC7047000000D0F0B594460025140E24
:1053D00001D112020835140F01D112010435940FC6
:1053E00001D192000235D40F01D152000135D40B06
:1053F0000134254F7C66254C3C660E0C93B2FFE7CA
:10540000FFE7FFE73C6F6643360C7703BE46734306
:10541000DF0B5B04C01AB941130C7343DB18C91AC4
:10542000CE086643360CB64493B273431F0F1B017C
:10543000C01AB941130C73431F0B1B05C01AB941A5
:10544000860D8F023E436643360C092D24DB520A3B
:105450007243801A7703460A6643360C16235B1B99
:10546000DE40DF40BF1964466643821B7046043548
:1054700006330100D940A840C01900D30131A2422F
:1054800006D20023F0BD0000000000D0FFFFFFFFA8
:10549000121B0130F3D3F1E709277F1BFE4064465E
:1054A000A2B27243801A00D20139220C7243130C4B
:1054B0001204821A99410B0070460435133701001B
:1054C000F940A840801900D30131002B02D1A2423B
:1054D0000AD2F0BD013000D30131121BFAD2013BD8
:1054E000F8D1A24200D2F0BD013000D30131121B2D
:1054F000F7E7F0B51C0C00D080E00CB400251C0AC6
:1055000004D11B02160E3343120208351C0B04D1C2
:105510001B01160F3343120104359C0B04D19B0071
:10552000960F334392000235DC0B02D192185B4197
:1055300001351C00971864410134464F7C66464C87
:105540003C660E0CFFE7FFE7FFE7C0463C6F664393
:10555000360C7703BE4697B27743C01B00D20139A1
:10556000C01B00D201399FB27743C91BC91B170C5E
:1055700077437E04FF0B801BB941CE086643360C8F
:105580000C2D33DBB644120B1F053A431B0B97B2AD
:105590007743C01B00D201399FB27743C91B170C58
:1055A00077433E043F0C801BB941860D8F023E437A
:1055B000664329277F1BFE400C3D7746AF40BF194D
:1055C00030BCA2B2ABB272437343801A9941220C31
:1055D0007243130C1204801A994102000B00013728
:1055E000001BA941F9D2781E0021F0BD0C277F1BBA
:1055F000FE4077467F0BAF40FF19E0E700245D1CBB
:1056000007D0144F7D663966FFE7FFE7FFE7FFE746
:105610003C6F95B29EB265436643401BB141150C89
:105620001E0C6543664336042F0C3E432D04401B7D
:10563000B141994204D202000B0020000021F0BDCC
:1056400001D19042F7D3801A994101349942F2D3A3
:10565000F6E70000000000D0FFFFFFFF4840414098
:10566000484018B41B4B5B68FC46019308BD04DF3F
:105670003759001018B4174B1B68FC46019308BD3E
:1056800000DF415900109446134A926F920809D2E4
:10569000624618B40F4BDB68FC46019308BD0CDF73
:1056A000F95B00100C4AF0B5146E556E576F166F0B
:1056B0006246FFF7EEFF084A14665566576716679D
:1056C000F0BD18B4034B9B68FC46019308BD08DF8E
:1056D0009D5A00104C8C0220000000D0FFB55040B5
:1056E0004240504059404B40594000E0FFB5154FF3
:1056F0004C00640D03D0BC4204D10C0314D800202C
:10570000090D09055C00640D03D0BC4204D11C03E3
:105710000AD800221B0D1B0501264B4009D44B4023
:1057200003D58B4200D18242FFBD9942FCD1904209
:10573000FFBD0B43DB1803431343F5D0C94349189E
:10574000FFBD0000FF07000000B5FFF7CFFF80415D
:1057500000BDC04600B5FFF7C9FF01D9002000BD5C
:10576000012000BD00B5FFF7B9FF01D9002000BD41
:10577000012000BD00B5FFF7B1FF804100BD012051
:1057800040054A00121804D85A00121801D8002007
:10579000704701207047002070470000002100285A
:1057A00005D17047C1174840401AFAD0C90713B550
:1057B000064B1B6898470CBC441CA2401005120BFA
:1057C0000349091B09051943114310BD4C8D0220E3
:1057D0001F04000010B54C00620D8023D218DB00BE
:1057E000D21A5B057E2A10DD9E3A13DACC17090324
:1057F000490819435242D140640001341532202A2D
:1058000005DAD0400843604310BD002010BD0846B3
:10581000604310BDC80FC018013810BD18B4044B48
:105820005B6AFC46019308BD24DFA95D00100000FF
:105830004C8C022070B513231C78012C14D0012C41
:1058400014DC022C02DC1F4A1F4B9A641F48FFF72E
:1058500071FC1F4B186070BD99001A481A4A885095
:1058600001331F2BF8D9EAE70023FAE71948FFF7BD
:1058700069FC05001848FFF765FC023803789B00B7
:105880007F2B19DD802229000F4800F007FC022C35
:10589000D7D1124B1A88B5231B029A4209D1104B5B
:1058A0001A88104B9A4204D10F4B1A880F4B9A4218
:1058B000C7D00020FDF750FF0D4B0E4A32210E4895
:1058C000FDF7B0FEFD5800104C8C02204C33000058
:1058D0004C8D022053440000534600005438000011
:1058E000D8380000494600009C38000059460000A6
:1058F00070A4001018A50010D0A4001007B56046D1
:10590000002800D100BE01880A0A0230DF2AFAD13D
:10591000C9B2820804D3028840880004104300E022
:105920000068024A5050039007BD00004C8C0220D2
:105930000FB403BC0CBCF0B50124E407634000E0E5
:10594000F0B50C0DCF0F661E3605891B640503D319
:10595000C943404200D30131640D03D0661CF60AEE
:1059600007D0E41B00207F00791C89078912803C46
:1059700024031D0DDF0F6E1E36059B1B6D0503D323
:10598000DB43524200D301336D0D03D06E1CF60A87
:1059900007D0ED1B00227F007B1C9B079B12803DE4
:1059A0002D032F1B661B58D4A446202E46DA203721
:1059B0001400BC401D00BD40F24033412A43801812
:1059C0005941CB0F05D0C943C04300226442504126
:1059D000514162464D0D28D10D0D07D100281FD031
:1059E000241940414941013A0D0DF9D0640006D314
:1059F000013000D30131002C01D140084000013AB0
:105A00000BD4941CE40A04D112051144DB07194499
:105A1000F0BDD907204B194300E0D9070020F0BDA5
:105A20000029DDD1002CDBD1F0BD0132C6074008D2
:105A3000CD0728434908002EE1D0D9E73C2E29DACA
:105A4000203E40371400BC4000D00124F2401443F3
:105A50001A00BB401C43D317ACE7AC46202F08DA32
:105A600020360400B4400D00B540F84039412843C9
:105A7000A5E73C2F0CDA203F40360400B44000D0AC
:105A80000124F84004430800B1400C43C117EAE781
:105A900010001900002494E70000F07FF0B50C0D11
:105AA000661E3605891BE60A6405640D02D0651C76
:105AB000ED0A04D0002001210905803C2403A446FE
:105AC0001C0D671E3F05DB1BE70A6405640D02D051
:105AD000651CED0A04D0002201231B05803C240331
:105AE0007740644497B484B296B27443070C7E4303
:105AF000150C6F4380B26843361802D301200004AE
:105B00003F183004350C00197D41844688B29AB2A2
:105B100050430C0C62431F0C7C438EB27E4392199F
:105B200002D301263604A4191604170C361867414F
:105B300001BC81B29AB25143040C62431B0C5C431A
:105B400080B25843121802D3012000042418100414
:105B5000130C401863412D185E410020474106BCDC
:105B600088B293B258430C0C6343120C544389B26D
:105B700051435B1802D301210904641819041A0C5B
:105B8000091862416D1856410020474118BCF902BE
:105B9000720D1143F0026A0D1043ED020A0D03D19C
:105BA0006D1940414941013B124E9B1B7600B342A7
:105BB0000ED26D0007D30130002671416646354391
:105BC00001D1400840001B05C918E4072144F0BD7D
:105BD0000BDA013306D1013004D101314F0D01D070
:105BE0004908F2E7E1070020F0BD01363105002049
:105BF000EBE70000FF030000F0B51C0D671E3F053A
:105C0000DB1BE70A6405640D02D0661CF60A04D0AB
:105C1000002201231B05803C2403D0252D060026ED
:105C2000F6432E661E096E66CE0FF619B44649007D
:105C30004F0D02D07E1CF60A03D000200021403F09
:105C40003F033E1BB600B444013F7F05C91B490812
:105C50002E6F013676089C02950D25437543ED1392
:105C60007543AD1301356D10F603761B0CB4CC02F1
:105C7000450D2C43A2B2B3B25A43270C7B43350CDB
:105C80006F43A4B26C431B1902D3012424043F19AF
:105C90001C041D0CA4187D4124196D41009A91B279
:105CA000ACB26143170C7C432B0C5F4392B25A4356
:105CB000A41802D301221204BF182204230C521884
:105CC0007B41019C6C431B19520ED9010A434401CC
:105CD000A01A81B2B2B2514303145A43360C734333
:105CE00087B27743D617D21900277E4136049B1915
:105CF0001704160C7F185E417316ED18F301002689
:105D000080337541A90F06D16400690AE8055B0A72
:105D1000184309D22FE00422944480337541A90A24
:105D2000A8059B0A184326D3404149412404009A00
:105D3000019B0D005543641B4343E41A95B286B2A0
:105D40007543170C7E43030C5F4392B25A43B61857
:105D500002D301221204BF183204330C52197B41C2
:105D600052429C41002C02D4002201305141400893
:105D7000CA071043490802B06246D7079210084B81
:105D8000D218084B9A4203D212058918C919F0BDDE
:105D90000020002A01DC3900F0BD01331905F5E7C8
:105DA000FD030000FE070000002200B5203200F0D5
:105DB00004F8080000BD000000220B150AD410B53D
:105DC000944600F031F81414013400DA0021CB17A6
:105DD000144C20470020002170476244343A0CD410
:105DE0000C2A07DA04009140904052422032D440FD
:105DF000214310BDD843D94310BD203207D40C46EF
:105E00009440524220321141D040204310BD08003E
:105E1000C917203203D452422032104110BD18005D
:105E2000190010BDDB5D00100A0DCC0F531E1B05C1
:105E3000C91A520503D3C943404200D30131520D60
:105E400003D0531CDB0A07D0121B00206400611C26
:105E500089078912803A1203014BD21A7047000059
:105E6000FF03000051434343C9188C46110C83B211
:105E70004B4310B4040C614392B280B2504362436E
:105E80001C041B0C001910BC59411304120CC0183F
:105E90005141614470470000484041404840002360
:105EA0009C46114B5B68184700239C460E4B1B68B1
:105EB00018470E4A936F9B0804D200239C460A4B56
:105EC000DB681847F0B5146E556E576F166FFFF705
:105ED000F4FF064A1466556657671667F0BD00233F
:105EE0009C46014B9B681847508D0220000000D053
:105EF000491A002808D1084670470000C10FC90799
:105F000000D54042002817D0F44603B40B4B1B6861
:105F1000984706BC81409E384042803107D20B062C
:105F200007D04900490AC0051043084360470130C3
:105F3000F8E7490A8902F5E7704700004C8D022016
:105F400000239C46014B5B6A18470000508D0220DD
:105F500070B513231D782A48FFF7F4F80400012DCB
:105F600011D0012D09DDA31E1B789B007F2B40DD86
:105F700080222100234800F091F82348FFF7DAF847
:105F8000224B186070BD542201001E4800F086F8B4
:105F90001F4B1A881F4B9A421CD1A7239B011A88BA
:105FA0001D4B9A4216D11D4B1A881D4B9A4211D196
:105FB0001C4B1A8894239B019A420BD11A4B1A88C6
:105FC0001A4B9A4206D11A4B1A681A4B9A4201D1BF
:105FD000152307E01848FDF7BFFB99001748094A49
:105FE000885001331F2BF8D9144A064B1A62DA6124
:105FF000B7E7134B134A42211348FDF713FBC04682
:1060000053460000508D02204C3300004C8D02207E
:10601000EE290000C40F0000C20D0000962B000006
:10602000C0B50000182B0000CC2A000010B50000FD
:10603000FC2C000051ED8764B09D00104D600010F5
:106040002CA50010A4A5001060A5001007B560469F
:10605000002800D100BE01880A0A0230DF2AFAD1E6
:10606000C9B2820804D3028840880004104300E0CB
:106070000068024A5050039007BD0000508D022076
:1060800001480421014B1847D0040020555100104D
:10609000014B1B6818470000D0040020014B5B68CF
:1060A00018470000D004002010B5030008001100BC
:1060B0001B68984710BD0000F8B507000D001600DA
:1060C000437C002B02D0002400200CE00368110068
:1060D000280098472DE03B7C10E0022115483B68E2
:1060E0009847601C0134B44214DA002CF3DD2B19FC
:1060F000013B1B780D3B5A425341DBB22A5D0A2A11
:10610000F0D1002BEED1A042E7DA211A28183B6823
:106110009847E2E7B04203DA311A28183B689847FB
:10612000002E06DDAD19013D2B780D3B5A4253413F
:106130003B74F8BDA4A6001070B505000368002BE1
:1061400016D00C4B1C6805E0290004C92000FFF79D
:10615000B3FFE468002C09D02368002BF9D0064B6C
:106160001B68002BF0D0A342F3D1EDE700232B6096
:1061700070BDC0467C8702208087022070B5050074
:106180000C000B68802B05D021684B1C2360641821
:10619000257170BD0800FFF7CFFFF5E7F0B583B0BC
:1061A00007000E000092019328E0A368002B04D0A2
:1061B000310038009847002827DCE468002C06D01E
:1061C000134B1D68002DF0D0A542F6D1EDE701205C
:1061D0000021FCF7D9FE0099019A0E4B5B6A9A42A6
:1061E00009D80C48806A88420BD29A4201D0012318
:1061F00002E0002300E00023002B04D1064B1C68C2
:10620000DCE70123F8E70120404203B0F0BDC046BF
:1062100080870220004005407C87022010B582B0B4
:10622000D0231B0600241C5701A9074803F06CF972
:10623000002806D1019B9C4203D0034803F074F967
:10624000012002B010BDC0462805002010B502484C
:1062500003F042F910BDC04628050020F0B5CE4637
:10626000474680B583B006000D0090461C00FFF73E
:10627000D5FF81466B1C05D0002C08D0194F1A4B56
:106280001C6807E0300003F0EDF80500F4E7174F55
:10629000F5E7E468002C17D02368002BF9D0144BE5
:1062A0001B68002B01D0A342F3D12A00310020004B
:1062B000B8474346002BECD06B46D91D0A230B7020
:1062C00001222000B847E4E74B46002B07D16B1EA4
:1062D0009D41E8B203B0C0BCB946B046F0BDFFF77F
:1062E000B5FFF4E7A96000107C870220B9600010B8
:1062F0008087022010B582B004006B46D81D047060
:10630000012300220121FFF7A9FF200002B010BDE8
:10631000094A01E00C331A001368002B08D08342AD
:10632000F8D1002907D1C36813600023C36002E0DD
:10633000002900D0106070477C87022010B5064B02
:106340001C6801E09847E468002C03D06368002BC8
:10635000F8D1F8E710BDC0467C87022070B5050073
:1063600003F080F804000023012201002800FFF759
:1063700075FFFFF7E3FF200070BD000070B5A2B00D
:1063800004000E00FFF74AFF05008422002101A847
:10639000FFF77EFE3300220001A90848FEF7B2FE97
:1063A000040001A8FFF7C8FEFFF7C8FF002D02D1C7
:1063B000200022B070BDFFF749FFF9E77D610010B2
:1063C0000FB400B583B004A901C90191FFF7D6FF4E
:1063D00003B008BC04B0184710B500F073F910BD45
:1063E00030B583B004000025FCF7AEFD02000B1EA3
:1063F00016DB12196B41994202D804D1904202D99E
:1064000001225242D317002B10DB012101A8FFF714
:10641000C5FE002802DB0FD001AB187803B030BDF9
:10642000094B0A4A3F210A48FDF7FCF8064B074A88
:106430003F210748FDF7F6F89221064B064A49002E
:106440000648FDF7EFF8C046C498001078A6001083
:10645000E0980010F099001090A600103CA60010E3
:1064600070470000014B00221A7070479A8E02207C
:106470004B79FF2B0CD18B79002B0BD1CB79012BD6
:106480000AD1082A0AD98A78054B1A70092000E037
:10649000002070470020FCE70020FAE70020F8E722
:1064A0009A8E02200120704770B504000D00034849
:1064B000FEF740FE030029002000984755420000E7
:1064C00010B5002926D1117953791B020B431249CB
:1064D00009788B4201D0002010BD5378012B03D0E6
:1064E000022B10D00020F7E79178D3781B021943D4
:1064F000DB0503D54B0A0120984000E000207F23F4
:106500001940FFF7D1FF642200210020FDF732FD82
:106510000120E1E70120DFE79A8E022001230370CA
:1065200000487047A8A6001010B50B784878000204
:1065300018438A7812041043CB781B060343962233
:10654000D200934200D010BD00210800FFF7ACFF3D
:1065500030B583B005000C0001A9184802F0D4FF43
:10656000002808D1D0231B061B68019A9A4221D02B
:10657000124802F0D9FF002001F01AFE002807D1CE
:10658000032464420D4802F0A7FF200003B030BD91
:10659000002001F02FFE002802D103246442F1E71D
:1065A00022002900002001F031FE041EEAD103245C
:1065B0006442E7E703246442E7E7C0465C8E0220BA
:1065C00010B50021054802F09FFF002800D110BD42
:1065D00001F086FB014802F07FFFF8E75C8E0220A5
:1065E000F0B5C64600B582B080460D0001A92E4820
:1065F00002F08AFF002808D1D0231B061B68019AED
:106600009A420FD0284802F08FFF002001F0D0FD01
:10661000002847D1254B00200021186059602248EE
:1066200002F05AFF02B080BCB846F0BD01F058FB42
:10663000002001F0FFFD002001F0BAFD0028EED09F
:10664000002001F079FE00281DD0AC42E7DA2E1BB5
:10665000002001F071FE0200864200DC3200002AB8
:10666000E4D043461919002001F04AFE060001F06B
:1066700037FB002001F0DEFDA419FCF765FC0B4B95
:1066800018605960E1E7FCF75FFC084B1E685F6823
:10669000074A002392197B419942C0D8D5D1904234
:1066A000D3D9BCE70024D0E75C8E02200081022011
:1066B00020A1070010B51F20FDF7EAF9FA2080009D
:1066C000002110BD70B584B0244B1B7802F07AF81D
:1066D00023491F20FDF7ECF901211F20FDF7D0F918
:1066E0002048FCF759FDFCF7A3F90600FCF72CFC49
:1066F00004000D1E20DBFA229200002312196B41C8
:10670000994202D804D1904202D901225242D317B1
:10671000002B17DB01210291002101911249009108
:106720003000FCF79BF90400631E9C41E4B2002892
:106730000ED1200004B070BD0C4B0D4A3F210D4816
:10674000FCF770FF094B0A4A3F210A48FCF76AFF31
:1067500001210948FFF7DCFDEBE7C04614AF00104C
:10676000C16500105C8E0220B5660010C498001050
:10677000E0A60010E0980010E004002000487047F8
:1067800078A700100048704724A7001010B5040037
:10679000154B1B78002B0ED0002C11D1134B144A33
:1067A0005A80012301335B001BB2C02292001343C5
:1067B0000E48038010BD11210B4802F0D7FBEBE718
:1067C000052C0ED8A4000B4BE4580023122BE9D85B
:1067D000E25C002AE6D00133590004484252DBB2A1
:1067E000F4E70020E6E7C0467C8E022044870220C2
:1067F000090400008CA7001002007F201040D2097D
:10680000400080184001014BC01870478487022067
:1068100010B582B001AB074A1A80002406E001AB34
:10682000185DFFF7E9FF0123C3700134012CF6D98D
:1068300002B010BD0080FFFF10B5838B3F333F22B5
:106840009343022915D0124C2268C260D3182360EA
:106850009C0610D10F4C6240634080246401A34227
:106860000FD88906114380231B061943436819601A
:1068700010BD5B00E7E7084B084A54210848FCF7C5
:10688000D1FE084B054A56210548FCF7CBFEC04611
:106890002C8C022000001050A4A70010BCA80010EF
:1068A000D4A7001028A80010F8B505000E001400A9
:1068B000FFF7A2FF7F232B40EF0985707A427A41D0
:1068C00042700022C27086838477012F0DD0DA00D7
:1068D00012498C4662448260826800211160002B5C
:1068E00009D143600E4BC360F8BDDA000D498C46F8
:1068F00062448260F0E7012F09D0013BDB000A4AC5
:106900009446634443602100FFF796FFECE7013BA8
:10691000DB00064A944663444360F4E78400105069
:1069200000011050800010500C0010500800105052
:1069300010B5002308E00133DA00002108481150A7
:10694000844662445160DBB20E2BF4D9F0229200EF
:1069500000210448FFF79CFB034B044A1A6010BD5A
:1069600000001050C48702202C8C0220800110509F
:10697000F0B5CE46474680B583B01D4B9F6D0024D1
:10698000012603E0B74376000134E4B2002F29D09A
:106990001F2C27D83E42F6D0164B9E6563089946B9
:1069A0000123634001221A4090464B465D00454456
:1069B0006D01114BED18280000F0ACFA0028E1D071
:1069C0004B465B0043445B010B4AD3189A8A997883
:1069D000012300930023002000F00AFE280000F0AD
:1069E00009FACFE703B0C0BCB946B046F0BDC04617
:1069F00000001150003011508487022070B52B4ADE
:106A00009823D45880235B0225001D401C420AD1E4
:106A1000E30616D4E30419D4630429D4230433D43D
:106A2000A5423ED170BDFFF7F3FE012220490020B0
:106A300000F0C4FD1F4B802292021A6580256D0272
:106A4000E6E710231D43FFF793FFE3E780235B0195
:106A50001D43164B00221A60FFF76AFF0122002136
:106A6000002000F096FD134B802212031A65D3E735
:106A70008023DB011D4301220421002000F076FD6C
:106A80000C4B10221A65C9E780231B021D4301220B
:106A90000521002000F06AFD064B802212011A65D4
:106AA000BEE7290061400448FCF756FE0000115083
:106AB00000001050003011505CA8001070B50C00A0
:106AC0001500FFF799FE2A00210000F0FFF970BDC4
:106AD00010B5002804D101210520FCF7D1FF10BD1D
:106AE000B921034B034A49000348FCF79BFDC0460C
:106AF00070A80010ACA80010D4A7001010B5002892
:106B000005D1002200218020FFF7D8FF10BDBF2152
:106B1000024B034A49000348FCF784FD70A80010AB
:106B20009CA80010D4A70010024B80225202DA6405
:106B30007047C0460020115070B5041E25D100F0EA
:106B400033F9154D0C23AB6714490520FCF7B0FF52
:106B5000402200211248FFF79BFA0022402100202A
:106B6000FFF7A2FE002240218020FFF79DFEFFF7E5
:106B7000DFFE01232B6480239B05EB649023094AED
:106B8000EA502000FFF7D0FF70BD4E21064B074AA8
:106B9000FF310748FCF746FD00001150FD69001069
:106BA0008487022010D0010070A80010D0A8001027
:106BB000D4A700100B785B0602D14B78052B00D0D0
:106BC00070478A78014B1A60FAE7C04600001150FE
:106BD00010B50C0000280DD10A794B790721194016
:106BE00009021143E2789207920FA078FFF75CFE4A
:106BF000012010BDD621034B034A49000348FCF78E
:106C000011FDC04670A800108CA80010D4A7001079
:106C100010B5FFF78DFE10BD10B50400080011007F
:106C20001A00002C03D1FFF749FF012010BDBC2141
:106C3000024B034AFF310348FCF7F4FC70A8001034
:106C40007CA80010D4A7001010B508004B0605D191
:106C5000CB09012B0AD00222054B9A66FFF7CCFD27
:106C600080221201002100F0CBF810BD0122F3E7D1
:106C70000020115010B508004B0600D110BDFFF7E1
:106C8000BBFD0023C3700022014900F0B9F8F5E70D
:106C9000FFF7FFFFF8B504000F00438A828B1E1C2C
:106CA000934200D9161CB6B29B1B63828025ED006F
:106CB0003543E378002B13D0802292011543012243
:106CC0005340E3706378002B0CD0638A002B02D111
:106CD0008023DB011D43002F00D02D042800F8BDC8
:106CE0000022EBE7B801E3689C4660443200A169EA
:106CF000FFF7D4F9A3699C466644A66180231B0272
:106D00001D43E2E770B5040083681B68002900D0CA
:106D10001B0C9D05AD0D6278002A11D11B0409D40E
:106D2000A38A5B19A382A38BAB4201D900236382A0
:106D3000280070BD0E4B0F4AD7210F48FCF772FC9C
:106D40001B040ED58901E3689C4661442A00A069B2
:106D5000FFF7A4F9A38A5B19A382A3695B19A36156
:106D6000E1E7064B034ADE210348FCF75BFCC04623
:106D7000DCA80010FCA90010FCA8001050A900100D
:106D800010B5040083681B680021FFF7BBFF636830
:106D90001B685B0002D5A38B834200D010BD01218C
:106DA0002000FFF7AFFFF9E710B580235B040C4A22
:106DB00013600C4A13600C4B9A6880235B04934366
:106DC000F9D10A4C9C2200212000FFF761F98022B2
:106DD000520100210648FFF75BF90923636710BDE4
:106DE00000E0004000F0004000C0004000001150F2
:106DF0000000105000230374438283828361704734
:106E000010B5002902D083681B681940002A0FD0F2
:106E1000114353050CD5826813685B050BD40B4BEB
:106E20000B401360FFE7FFE7FFE7FFE7FFE7FFE740
:106E30008368196010BD83787F211940DB099B00AE
:106E4000034A9A580348FCF787FCC046FFFBFFFF44
:106E5000F404002070A9001070B5040043681E6897
:106E60000021FFF717FF80256D010543144B1B6CB4
:106E70009B0704D4A378DB0914D1013300E000237D
:106E8000628A002A01D0002B0ED00E4B1E408023B8
:106E90009B053343626813602A0000212000FFF73E
:106EA000AFFF70BD0023EBE701212000FFF7F2FEEA
:106EB0000543054B1E40A023DB053343EAE7C046EC
:106EC00000001150FFFFFFAFFFFFFFDF70B50400B0
:106ED0000D001600037C002B09D166820023A382DB
:106EE00001332374A5612000FFF7B6FF70BD8378DE
:106EF0007F211940DB099B00044A9A580448FFF798
:106F00005FFA2000FFF776FFE7E7C046F4040020B1
:106F100090A9001070B50400057C002D06D0FFF785
:106F20002FFF638A002B08D1280070BD81787F2352
:106F30001940044A0448FCF70FFC2000FFF78CFFBF
:106F40000025F1E7F4040020C8A9001070B5050081
:106F500000240EE063001B19DA00184B1B689B1815
:106F600002E0230010E000235B682800984701340A
:106F7000E4B2134B1B78A3420ED3124A002AF0D07E
:106F8000A342E7D8E31ADBB2002BECD15A00D218A7
:106F9000D2000D4B9B18E7E70C4C53220021200038
:106FA000FFF776F8E01C1022FF21FFF771F82000B0
:106FB00013302022FF21FFF76BF870BD648102209F
:106FC000908E02201D65001044AB00109C840220AE
:106FD00010B5FFF7BBFF01F02BF810BD70B5050031
:106FE0000C001600C86801F02DF8E368320000219B
:106FF0002800984770BD0000F0B5DE4657464E4663
:107000004546E0B583B081460139C8B2FFF7BAFB07
:10701000002803D043789846022B0CD0564A574993
:107020005748FFF7CDF9002003B0F0BCBB46B2468D
:10703000A946A046F0BDC5796A11012351491A40FD
:1070400014010A781026B24322430A70AD112B4076
:107050005B01D2B22024A24313430B70070009370F
:107060008178C3781B020B4382469A4463E0FB7825
:107070009B463B78FF1865E0434A40494048FFF78C
:107080009FF90020D0E766003619F3003F4A1668E2
:10709000F61802E0230017E000262A0039004846CF
:1070A000B36898470190082801D9854214D2013469
:1070B000E4B2374B1B78A34239D3364A002AE9D0D1
:1070C000A342E0D8E31ADBB2002BE5D15E00F3184F
:1070D000DB00314EF618E0E75B46012B10D00022B2
:1070E00093451AD9BB789B18DBB22649C918C978D1
:1070F000FF290BD12349CB18DC700132D2B2EFE764
:10710000B268264B9A42EAD1C346E8E7244A1B49B3
:107110001B48FFF755F9002086E71A482300019D18
:107120002A003900133001F0BBFBAC466744184B12
:107130001B78A3420ED3574514D27B780B2B96D0E5
:1071400001239B467B78042B96D15346DD1BADB2C1
:107150000024AEE7F322920008490948FFF730F90E
:10716000002061E70F4B002B03D000E000BF01209F
:107170005AE7012058E7C0467B0300000CAB001023
:107180000CAA00109C840220960300006481022057
:10719000908E02201D65001044AB00105584001035
:1071A000BD0300000000000070B505000C00CB78A6
:1071B00088780F2B54D89A002F498A589746FFF7A2
:1071C000DDFA020012232100280000F0DDFE48E075
:1071D0002A4B002B46D000E000BF02008178C37824
:1071E0001B020B432100280000F0CEFE39E0022BE9
:1071F00010D0234B002B37D000E000BF0200002A44
:107200000CD09178D3781B020B432100280000F0AA
:10721000BBFE26E0FFF7B6FA0200F0E7194A1A496A
:107220001A48FFF7CDF800201BE0237961790902A5
:107230001943FFF7ABFA021E18D00378210028008B
:1072400000F0A2FE0DE0124B002B11D000E000BFB9
:10725000021E0FD003782100280000F095FE00E008
:10726000002070BD0020FCE70020FAE70020F8E7CE
:107270000020F6E70020F4E724AA00100000000038
:107280000000000014040000F4AA00100CAA001072
:1072900000000000024B5878431E9841C0B270476E
:1072A0009C840220024B18784007C00F7047C046EC
:1072B0009C840220014B18787047C046918E0220B2
:1072C00070B50500274B1878002800D070BD5322F8
:1072D00000212548FEF7DCFE244C2000FBF75CFF74
:1072E000234B1C60234C20001C30FBF77BFF20004D
:1072F00001F0F0FD204B1C60204B002B04D02048F7
:10730000FFF70CF91F4B186000240DE063001B19F8
:10731000DA001C4B1B689B1802E023000FE00023DF
:107320001B6898470134E4B2154B1B78A3420ED377
:10733000124A002AF1D0A342E8D8E31ADBB2002BAC
:10734000EDD15A00D218D2000F4B9B18E8E7280065
:10735000FFF7F2FB2800FFF7BBFB024B01221A707C
:107360000120B3E7918E02209C84022054840220E5
:10737000F0840220FC040020F48402201D6500102B
:10738000908E02206481022044AB001030B585B09D
:1073900004004378042B00D196E038D8022B62D049
:1073A000032B00D0B9E06D4B1B785B0700D483E062
:1073B0006A4A137804218B4313700C22002101A820
:1073C000FEF766FE23786A46137105235371644BFA
:1073D0001C68E269EFF3108172B61368002BFCD0D1
:1073E000BFF35F8F216201A9200001F038FDE2693F
:1073F000236ABFF35F8F0021116083F31088002898
:107400005AD1A82257495848FEF7DAFF54E0052B15
:1074100000D082E0514B1B78DB074DD54F4A1378E3
:1074200004218B4313704E4B1D68EA69EFF3108102
:1074300072B61368002BFCD0BFF35F8F2962210066
:10744000280001F00CFDEA692B6ABFF35F8F002171
:10745000116083F3108800282ED1A82241494248A8
:10746000FEF7AEFF28E03D4B1A7801218A431A70DF
:107470001A7801318A431A7000225A701A78023140
:107480008A431A70364B1D68EA69EFF3108172B6B1
:107490001368002BFCD0BFF35F8F29622100280006
:1074A00001F0DDFCEA692B6ABFF35F8F00211160F8
:1074B00083F31088002801D005B030BDA8222949E7
:1074C0002948FEF77DFFF7E7244B1B78DB07F3D550
:1074D000224A137804210B431370214B1D68EA697B
:1074E000EFF3108172B61368002BFCD0BFF35F8FEF
:1074F00029622100280001F0B2FCEA692B6ABFF37F
:107500005F8F0021116083F310880028D4D1A82256
:1075100014491548FEF754FFCEE7114B1D68EA6980
:10752000EFF3108172B61368002BFCD0BFF35F8FAE
:1075300029622100280001F092FCEA692B6ABFF35E
:107540005F8F0021116083F310880028B4D1A82236
:1075500004490548FEF734FFAEE7C0469C8402208C
:10756000F4840220E4AA00100CAA001070B584B0C4
:1075700006000D0014000C22002101A8FEF788FD72
:107580006B461E715D71210001A8FFF7FFFE04B07C
:1075900070BDF0B585B007000E00150001AC0C22DF
:1075A00000212000FEF774FD27700123637026710F
:1075B00029002000FFF7EAFE05B0F0BD70B584B0E9
:1075C00006000D0014000C22002101A8FEF760FD4A
:1075D0006B461E7106236A4653710822290002A8D1
:1075E000FEF75CFD210001A8FFF7D0FE04B070BDDE
:1075F000F0B5CE46474680B585B080460F001600F0
:107600001D000CAB1B78994601AC0C220021200018
:10761000FEF73EFD434623700723637027710396F0
:10762000657149462000FFF7B1FE05B0C0BCB94600
:10763000B046F0BD70B506000D008B7870221A427E
:107640000DD10D4B9978280001F0D6F8041E0DD00D
:1076500029003000FFF7BCFA0400200070BD074A83
:1076600007490848FEF7ACFE0024F6E7064A04493D
:107670000448FEF7A5FEF0E79C840220C204000047
:10768000C0AA00100CAA0010C3040000F0B5D64632
:107690004F464646C0B581460C0017009846089BE9
:1076A0009A46002516E0184A18491948FEF788FE40
:1076B00000263000E0BCBA46B146A846F0BD154AE7
:1076C00012491348FEF77CFEF3E7099A13702378FA
:1076D000E4180135AF4214DD6378052BE3D1E1787E
:1076E0008907890F4145DED121004846FFF7A2FFF7
:1076F000061EE4D0A378DA09012AE6D052461370B8
:10770000E5E70126D5E7C0469C040000D0AA00109A
:107710000CAA00109D04000070B57F250D40CC0917
:107720006A001E4B9B181B193033DB78DB07DE0F1A
:10773000002B30D1194B9B181B193033DB785B07BA
:107740002AD4174B18680121494201F0E5FE6A006E
:10775000124B9B181B193033DB78DB0708D40F4B17
:107760009B181B193033DB785B0712D5002600E02D
:107770000026002E08D06D0008494D192C19303410
:10778000E37804221343E370054B186801F0A4FE6C
:1077900002E00126EDE70026300070BD9C84022047
:1077A000F084022070B57F250D40CC09154B186878
:1077B0000121494201F0B0FE6A00134B9B181B19CE
:1077C0003033DB78DB0708D40F4B9B181B193033A1
:1077D000DB785B0713D4002600E00026002E08D0DB
:1077E0006900094D6D182C193034E3780422934355
:1077F000E370044B186801F06FFE300070BD012685
:10780000ECE7C046F08402209C840220F0B5C64616
:1078100000B582B001937F250D40CE096F00174C53
:10782000E419A4193034E478E4071DD46F00134C34
:10783000E419A4193034E3780127BC4667463B437A
:10784000E370019BFFF7E8F9002813D16D000B4BA3
:107850005D19AE193036F37801229343F370F37853
:1078600003329343F37005E0054A06490648FEF7E4
:10787000A7FD002002B080BCB846F0BD9C84022069
:107880000A050000B0AA00100CAA001070B57F24F1
:107890000C40CD0962000C4B9B185B193033DB7830
:1078A0009B0700D570BDFFF7CFF96300064CE418C5
:1078B00064193034E37802221343E370E378012241
:1078C0001343E370EEE7C0469C84022070B57F242A
:1078D0000C40CD0962000C4B9B185B193033DB78F0
:1078E0009B0700D470BDFFF7C5F96300064CE41890
:1078F00064193034E37802229343E370E378013A69
:107900009343E370EEE7C0469C8402207F220A4046
:10791000CB09520003498918C9183031C87880074B
:10792000C00F70479C840220F0B5C64600B582B0F7
:1079300005000C00002000F085FB23786022134036
:10794000602B12D0402B17D02278D206D20E012AFB
:1079500000D1D9E0022A00D120E1002A1AD0002665
:10796000300002B080BCB846F0BDCC4ACC49CD480E
:10797000FEF726FD0026F3E7CB4B002B00D181E17B
:10798000180000F05FFB22000021280000E000BF8B
:107990000600E5E7202B0AD0002B00D07AE16378BF
:1079A000092B00D978E19B00C04AD3589F46237920
:1079B0000F2B00D968E1BE4AD318DB78BD4A002AF4
:1079C00005D0BD4A1278934212D39B1ADBB2002B2A
:1079D00000D05BE15900CB18DB00B849C918002979
:1079E00000D155E122002800FFF7F8FA0600B7E7BA
:1079F0005900CB18DB00B24A1168C918EFE7200024
:107A000000F026FBA1782800FFF778F8A84A137841
:107A100002210B4313700126A2E7A54B5B786A464F
:107A20000632137001232100280000F0ADFA012670
:107A300096E7A7789E4B5B78DBB2BB4205D09C4BA8
:107A40005B78002B09D1002F13D1994B5F70210077
:107A5000280000F07DFA012682E72800FFF7D8F819
:107A6000934EB37898462800FFF770FA4346B370F8
:107A7000E9E739002800FFF7BFFA061EE5D1914A71
:107A800087498848FEF79CFC6AE721002800FFF739
:107A90008BFB060064E7A278E3781B021343012BFB
:107AA00001D000265CE7824A137808210B4313704B
:107AB0002100280000F04CFA012651E7A278E37873
:107AC0001B021343012B01D0002649E7784A1378A3
:107AD00008218B4313702100280000F039FA012699
:107AE0003EE7734B1A785109920801230B4002219B
:107AF0000A4013436A4606321380022321002800FD
:107B000000F042FA01262BE723790F2B00D9DDE0A4
:107B1000674AD318D978674B002B05D0664B1B7882
:107B2000994229D3C91AC9B2002900D0D0E04B002C
:107B30005B18DB006149C918002900D1CAE02200A6
:107B40002800FFF74BFA061E00D009E723786022D1
:107B50001A4200D004E763780A3B012B00D9FFE604
:107B6000002000F06FFA63780A2B0CD02100280067
:107B700000F0EEF90126F3E64B005B18DB00504AFB
:107B80001168C918D8E76B469A1D0023137001339A
:107B90002100280000F0F8F90136E1E621797F2282
:107BA0000A40CE097020084220D152004048821875
:107BB0009219D27C3F48002805D03F480078824285
:107BC0001BD3121AD2B2002A1ED15600B218D2000C
:107BD0003A4EB618002B19D0002E00D17CE02200BE
:107BE00031002800FFF7FAF90600B9E6364A2C49B9
:107BF0002C48FEF7E5FB0026B2E65600B218D2008C
:107C00002F480668B618E5E70026E3E76378012BFE
:107C100012D0032B10D0002B01D00026A0E62800A4
:107C2000FFF774FE6B469A1D108002232100280086
:107C300000F0AAF9012693E6A778E27812023A4307
:107C400004D1012B1AD02800FFF720FE002E45D0CA
:107C5000220031002800FFF7C1F9002000F0F2F9FE
:107C6000134A3423D35CDB07DE0F002B00D077E60A
:107C70002100280000F06CF9012671E62800FFF7CA
:107C800025FEE3E700266BE6002669E6002667E6A8
:107C9000002665E6002663E6002661E67F02000016
:107CA00020AB00100CAA00100000000064AA001015
:107CB0009C8402201D650010908E022044AB0010B1
:107CC00064810220D302000033030000002647E64F
:107CD000002645E6002643E6002641E601263FE66B
:107CE00030B585B000F080FD002808D105B030BD6A
:107CF00001AC2078FFF76CF92279724B9A70724BC5
:107D00001C68E269EFF3108172B61368002BFCD097
:107D1000BFF35F8F216201A9200001F07AF8E269C8
:107D2000236ABFF35F8F0021116083F3108800285E
:107D3000DCD001AB5B78082BE1D89B00634AD358B9
:107D40009F4601AB1878FFF743F9614B002BD6D063
:107D500000E000BFD3E75B4B1A78012401210A43FE
:107D60001A703322995CA1439954995C0420814391
:107D700099540132995CA1439954995C8143995477
:107D800001AB187802A9FFF7CFFD0028B7D101ACED
:107D900020780021FEF758FF20788021FEF754FF5D
:107DA000ADE701AB19797F220A40CC095000454B61
:107DB0001B181B193033D8780125A843D870D87800
:107DC0000335A843D870002A1DD052003D4B9A18A5
:107DD0001219D37C3F4A002A05D03F4A12789342B9
:107DE00018D39B1ADBB2002B1BD15A00D218D20039
:107DF0003A4B9B18002B14D01C6901A84279039BB5
:107E00000078A0477BE701A84279039B007800F047
:107E10002DF974E75A00D218D200314B1B689B1819
:107E2000E8E7304A30493148FEF7CAFA5EE7254BA9
:107E30001B78DB0700D462E72D4B002B00D15EE7F7
:107E4000204B18780007C00F00E000BF57E71D4B1C
:107E50001B78DB0700D452E7264B002B00D14EE7FE
:107E600000E000BF4BE763001B19DA001C4B1B68E6
:107E70009B1802E0230014E000235B69002B02D072
:107E800001AA107898470134E4B2134B1B78A3423F
:107E900000D234E70F4A002AECD0A342E3D8E31A19
:107EA000DBB2002BE8D15A00D218D2000B4B9B1842
:107EB000E3E70024E9E7029B002B00D11FE70398CA
:107EC00098471CE79C840220F48402208CAA0010AE
:107ED000000000001D650010908E022044AB0010D1
:107EE000648102203702000038AB00100CAA001099
:107EF0000000000000000000F8B50500124B9F894B
:107F0000DE89B91B89B20B1C402900D940239CB2E1
:107F10000D4B1B785BB2002B08DB0021B74211D060
:107F20000A4A23002800FFF771FCF8BDB74201D1CF
:107F30008021F3E7044B996822000448FEF7AEF86D
:107F40008021EBE70022ECE7408402205C840220E1
:107F500070B506000C000B4D08222800FEF79EF8B5
:107F60000023AB60EB81AB810023E356002B06DBE3
:107F70008021002300223000FFF748FC70BD002163
:107F8000F7E7C04640840220F0B5C64600B58046FB
:107F90000C0016001D00234F08223800FEF77EF863
:107FA000BE600023FB81A379E179090219430B1C10
:107FB000A94200D92B1C99B21A4A9381A279E3797C
:107FC0001B02134319D0002901D0002E08D04046CF
:107FD000FFF792FF041E0AD0200080BCB846F0BD17
:107FE000732211491148FEF7EBF90024F4E77922D6
:107FF0000D490E48FEF7E4F9EEE70023E356002BA7
:108000000DDB8021002300224046FFF7FFFB041E0A
:10801000E2D17E2204490548FEF7D2F9DCE70021CF
:10802000F0E7C0464084022074AB00100CAA001098
:1080300010B5142200210248FEF72AF810BDC046F0
:1080400040840220014B18617047C04640840220E2
:1080500010B50100044C08222000FEF71FF8002391
:10806000A360E381A38110BD4084022070B50500A8
:108070001C00C909374B1B78DB098B4219D0002C37
:1080800010D1354B002B02D03249FEF793FD314B16
:108090001B69002B03D02F4A022128009847012496
:1080A000200070BDAB222D492D48FEF789F9002430
:1080B000F6E7284B1B785BB2002B07DB254B986853
:1080C000002844D022002749FDF7E8FF214AD38940
:1080D0001B199BB2D381916809199160D288934290
:1080E00001D03F2C28D81B4B1B69002B05D0194A07
:1080F000012128009847002814D0164B1B785BB24A
:10810000002B0DDB8021002300222800FFF77EFBDF
:10811000041EC5D1D82211491148FEF751F9BFE715
:108120000021F0E700212800FEF78EFD80212800C5
:10813000FEF78AFD0124B3E72800FFF7DDFE041EE9
:10814000AED1E32205490648FEF73AF9A8E7002434
:10815000A6E7C04640840220B56B00105CAB00105F
:108160000CAA00105C84022070B5040005001035D4
:10817000280000F03EFE3F2800D870BDE1780020C6
:10818000FFF7CAFA0028F8D0280000F032FE3F2896
:1081900008D996239B00E218E17840230020FFF7DE
:1081A00035FBEAE7E1780020FFF7FCFAE5E700009D
:1081B00010B50400FFF76EF800280CD10022002A49
:1081C00011D0B6239B0063430948C0180379DB072D
:1081D0000BD5012008E0FFF765F8002801D1012246
:1081E000EDE70022EBE7002010BD0020FCE7C046D1
:1081F0006881022010B5B6239B0058431030024B13
:10820000C01800F0DBFD10BD6881022070B5B623F8
:108210009B005843064BC51892B21030C01800F0AE
:1082200019FE04002800FFF79FFF200070BDC04624
:108230006881022070B50500FFF72CF8002804D1F2
:108240000023002B09D1002070BDFFF72BF8002878
:1082500001D10123F5E70023F3E7B624A4006C4322
:108260002834244BE4180434200000F0A7FD002833
:1082700001D10020E8E7B62292006A431D4B9B180B
:1082800099780020FFF748FA002801D10020DBE7A9
:10829000B626B6006E43A6239B009C466644154B4B
:1082A000F61840223100200000F0D4FD041E15D045
:1082B000B620800068430F4D2D18A97823003200A6
:1082C0000020FFF7A3FA002801D02000BCE7C82255
:1082D00009490A48FEF774F80020B5E7B620800087
:1082E0006843044D2D18A9780020FFF75BFA0020A1
:1082F000AAE7C04668810220A4AB00100CAA0010B7
:1083000070B50500B624A40044432834094BE41892
:10831000043492B2200000F0D8FD0600200000F0E6
:108320004DFD3F2801D8300070BD2800FFF782FFC7
:10833000F9E7C0466881022010B5B6239B00584378
:108340002830034BC018043000F053FD10BDC04668
:1083500068810220F0B5CE46474680B583B0B6228C
:10836000920000212848FDF793FE0026002E04D03D
:1083700003B0C0BCB946B046F0BD234FB624A4003C
:1083800074433D19FF236B71002398461F4AEA800E
:1083900001222A81AB72EB7208232B732100483132
:1083A000C919F833994620001030C019434600938C
:1083B00001334A4600F0C9FC21004931FF31C91997
:1083C00020002830C0190430012300934A4600F0F1
:1083D000BCFC92239B00E3189946B9444846FAF73F
:1083E000DBFE43466B624B46AB6294239B009C468C
:1083F0006444E4192000FAF7CFFE2C6443466B6412
:108400000136F6B2B2E7C0466881022000C2FFFF23
:1084100070B50025002D00D070BDB624A4006C43BB
:108420000B4EA01905220021FDF732FE200010306E
:10843000801900F04FFD2834A4190434200000F006
:1084400049FD0121200000F06BFD0135EDB2E1E7AF
:1084500068810220F0B583B006004B79022B68D109
:108460008B79022B69D10023002B08D00027002F25
:1084700013D08B783B700C780C19092519E0B624C1
:10848000A4005C432E4800198078002802D00133F4
:10849000DBB2E9E72A4FE719E9E78F2252002949C1
:1084A0002948FDF78DFF002544E021784D19ADB234
:1084B00064186378242B01D19542F6D9052B09D095
:1084C0006378042B02D163790A2B18D03800FFF7A8
:1084D0004BFE2FE021003000FFF7ACF8002806D05B
:1084E000A3787B7022785519ADB2A418E8E79922D9
:1084F000520014491448FDF763FF00251AE0217863
:108500004D19ADB26118BB1C0193FB1C00930223F3
:1085100002223000FFF7BAF8002802D00E35ADB2C3
:10852000D4E7A122520007490748FDF749FF00257B
:1085300000E00025280003B0F0BD0025FAE7C046A2
:108540006881022098AB00100CAA0010F8B5140046
:10855000127860231340202B00D07FE0444A00258E
:10856000002D00D07CE01678277963791B023B430D
:108570009E4206D00135EDB2B6239B009C46624474
:10858000EEE76378222B31D009D8202B11D0212B94
:1085900003D1002923D0012061E000205FE0232BDC
:1085A00005D1002949D002294CD0012057E00020F4
:1085B00055E0002903D0022908D001204FE00632FF
:1085C00007232100FFF7E0FC012048E0294B002BA6
:1085D00048D0911D2800FDF7A7FF01203FE006329B
:1085E00007232100FFF7D0FC012038E0002903D049
:1085F000022906D0012032E02100FFF7A9FC01206A
:108600002DE0A178E3781B020B4301201900014003
:108610000E005C08044013714B425941C9B22C3220
:10862000100000F07DFC144B002B1DD02200310007
:10863000280000E000BF012011E02100FFF788FCC6
:1086400001200CE00D4B002B10D0A378E17809023B
:108650001943280000E000BF012000E00020F8BD21
:108660000020FCE70120FAE70120F8E70120F6E707
:108670006881022029650010000000000000000051
:10868000F0B5D64600B582B001900F0000930024EB
:10869000002C0DD0002C19D1EB78BB421ED0AB784A
:1086A000BB4255D00124200002B080BCBA46F0BDC8
:1086B000B625AD0065433D4BED18EB78BB42E9D0E4
:1086C000AB78BB42E6D00134E4B2E1E7B022FF323E
:1086D00037493848FDF774FE0024E4E710239A4632
:1086E000AA4496239B00E9186B461A88504600F06E
:1086F000ECFB314B002B1BD06B79FF2B18D00026E5
:1087000000E00136009B9E4212D26A79AB19962195
:1087100089008C4663441B789A42F2D1504600F09F
:1087200060FB0028EDD16979200000E000BFE8E798
:10873000224B002B04D0504600F053FB002803D0FE
:108740002800FFF711FDAAE7200000E000BFF7E7CF
:108750001B4B002B02D0200000E000BF2000FFF7E1
:1087600069FD002801D001249DE728002C3000F08D
:1087700025FB002815D1009B002B14D09B0601D0AF
:10878000012490E7A9780198FEF7C6FF041E01D1E5
:10879000012488E7A978002300220198FFF736F822
:1087A00081E701247FE701247DE7C046688102203C
:1087B00088AB00100CAA00100000000000000000B0
:1087C0000000000010B50020FEF77AFD041E01D065
:1087D000200010BD292202490248FDF7F1FDF7E70C
:1087E000D0AB00100CAA001010B5FEF763FD0028F6
:1087F00000D0012010BD000010B502794479072394
:1088000023401B021A43C3789B079B0F022B16D0F1
:10881000032B2ED0012B01D0002010BD022904D043
:108820001C4B934204D30120F7E78023DB00F8E7D9
:10883000502219491948FDF7C3FD0020EDE7022930
:1088400003D0402A0ED80120E7E780239B009A42FC
:1088500001D10120E1E758220F491048FDF7B0FD92
:108860000020DAE75C220C490C48FDF7A9FD002046
:10887000D3E7022904D04023934204D30120CCE75C
:108880008023DB00F8E7632203490448FDF798FDE5
:108890000020C2E7FF030000BCAB00100CAA0010D0
:1088A00070B5002503E00E78AD19ADB28919954277
:1088B0000AD24C78052CF6D18E787A343440640094
:1088C0000419F609A355EEE770BD03008A1890B2AB
:1088D000884202D39A89904202D95A89801880B27C
:1088E000704710B503008A4204D8881A80B29C8968
:1088F000A04204D9891A89B25889081A80B210BDD9
:10890000838801E0C91A89B28B42FBD908007047FD
:10891000F0B583B00600019111001F00D41AA4B273
:108920009A4202D24389E41AA4B2B588A54205D27C
:108930002A003000FFF7D5FF30822C00002C02D136
:10894000002003B0F0BD39003000FFF7D9FF3168D7
:10895000F288504309180198FDF7A0FB0120F0E7C9
:10896000F0B583B0060093080CE00B784D782D022B
:108970001D438C7824042543CB781B062B4333609E
:1089800004313B005F1EBFB2002BEED10333100059
:1089900018401A4201D103B0F0BD00230193020038
:1089A00001A8FDF77BFB019B3360F4E7F0B5DE46E1
:1089B00057464E464546E0B583B005008A460CA9A9
:1089C00009788488E01A80B21C1B1419A4B2EE88BE
:1089D00007007743BFB27443A4B2A34673432C6825
:1089E000A0469844002908D001291AD003B0F0BC51
:1089F000BB46B246A946A046F0BD904205D372439D
:108A000041465046FDF74AFBF0E73A0041465046E2
:108A1000FDF744FB2968380050445A46FDF73EFBF9
:108A2000E4E7904206D3724392B241465046FFF7C4
:108A300097FFDBE703233A009A43914641465046AD
:108A4000FFF78EFF43464B4403213A000A400F4292
:108A500030D00421891A89B2081C594500D95846DA
:108A6000C7B2FF2101405846441AA1B28B460021EB
:108A7000019101A804E01A78027001300A00013364
:108A8000511EC9B2002AF6D1296804E00A780270A2
:108A900001301F0001317B1EDBB2002FF6D153469F
:108AA000019A1A605B46002BA0D05A465046FFF749
:108AB00057FF9BE72968F5E7F0B585B005000291FF
:108AC00003920AAA11880BAA17785C1AA4B28B42E7
:108AD00002D24289A41AA4B2AE88A64208D23200B9
:108AE00019002800FFF7FDFE2882298A89B2340088
:108AF000002C0DD0039B9C4200D31C002800FFF7E4
:108B0000FFFE03000097220002992800FFF74EFFA6
:108B1000200005B0F0BDF0B583B004000D001600D4
:108B20001F008069002803D00121494200F0F4FCB5
:108B3000E3899BB2228A019700923200290020002B
:108B4000FFF7BAFF0500218A89B202002000FFF773
:108B5000BCFE2082A069002801D000F0BDFC2800E6
:108B600003B0F0BD70B582B01600950809E00B683F
:108B700003701D0A45701D0C85701B0EC3700430F8
:108B800025006C1EA4B2002DF1D1032332001A403F
:108B90001E4201D102B070BD0B68019301A9FDF71F
:108BA0007DFAF7E7F0B5DE4657464E464546E0B556
:108BB00083B005008A460CA90878AC88E11A89B20E
:108BC0001C1B1419A4B2EE880F007743BFB2744384
:108BD000A4B2A34673432C68A0469844002808D04A
:108BE00001281AD003B0F0BCBB46B246A946A04645
:108BF000F0BD914205D3724351464046FDF74EFA0F
:108C0000F0E73A0051464046FDF748FA2868390037
:108C100051445A46FDF742FAE4E7914206D37243C3
:108C200092B251464046FFF79DFFDBE703233A002F
:108C30009A43914651464046FFF794FF43464B44C2
:108C400003213A000A400F422ED00421891A89B22A
:108C5000081C594500D95846C7B2FF210140584663
:108C6000441AA1B28B4651460968019101A904E05A
:108C70000A781A70013102000133501EC0B2002A76
:108C8000F6D1286804E00A78027001311F00013033
:108C90007B1EDBB2002FF6D15B46002BA2D05A46DA
:108CA0005146FFF75FFF9DE72868F5E7F0B5CE4630
:108CB00000B584B004008946151E039343D0406973
:108CC000002803D00121494200F026FCE789BFB209
:108CD000238A9BB2227A002A2AD1A288F91A89B261
:108CE0009F4202D26389C91A89B2531A9BB22E1CC1
:108CF0009D4200D91E1CB6B239002000FFF700FECD
:108D00000300039A0092320049462000FFF74AFF11
:108D1000320039002000FFF7D8FDE08160690028AB
:108D200001D000F0D9FB300004B080BCB946F0BDE2
:108D3000A688AE4205D8AA1BE5885543A9441F0062
:108D4000DAE72E00D8E71600EDE7F0B583B00500AE
:108D50000F001400019308AB1E7880231B029A4277
:108D600028D84069002803D00121494200F0D4FBF3
:108D7000A869002803D00121494200F0CDFB2F60F3
:108D8000AC80019BEB802E726400013CA4B2AC81EC
:108D9000E4436C810023EB812B826869002801D0B9
:108DA00000F09AFBA869002806D000F095FB01208E
:108DB00003B0F0BD0020FBE70120F9E710B5C3893F
:108DC0009CB2028A91B29B1A9BB28C4202D2428917
:108DD0009B1A9BB28288101C9A4200D9181C80B240
:108DE00010BD0300C0891B8AC01A43425841C0B25B
:108DF000704730B5C3899DB2018A8CB282885B1AF4
:108E00009BB2A54202D240891B1A9BB2D01A80B2F3
:108E100030BD70B504000D008069002803D0012129
:108E2000494200F079FBE28992B2238A9BB2290081
:108E30002000FFF76DFD0500218A89B282B2200073
:108E4000FFF743FD2082A069002801D000F044FB19
:108E5000280070BD10B50023FFF75DFE10BD70B592
:108E600004000D004069002803D00121494200F0B0
:108E700053FBE3899EB2228A91B29B1A9BB2B14204
:108E800002D962899B1A9BB2A2889A4202D1207AA7
:108E9000002817D031002000FFF732FDE288504350
:108EA00023689C4660442900FDF7F8F80122310050
:108EB0002000FFF70AFDE0816069002803D000F080
:108EC0000BFB012070BD0120FCE710B50023FFF76C
:108ED000EDFE10BD10B504004069002803D001214B
:108EE000494200F019FBA069002803D00121494242
:108EF00000F012FB0023E3812382A3885B00013B87
:108F00009BB2A381DB4363816069002801D000F03C
:108F1000E3FAA069002801D000F0DEFA012010BDBC
:108F200070B504000D004069002803D001214942BA
:108F300000F0F2FAA069002803D00121494200F0B4
:108F4000EBFA25726069002801D000F0C5FAA0692B
:108F5000002801D000F0C0FA012070BD10B5024811
:108F600000F034F810BDC046448C022010B5002932
:108F700001D000230AE0114B114A1F311148FAF7C2
:108F800051FB00240DE03732C25401334A1E9A428D
:108F90000FD90F2B0DD85A080B4CA25CDC07F0D46C
:108FA0000424224114000F222240092AEBDC303233
:108FB000EAE7C0180023037010BDC046DCAB001008
:108FC00028AC0010E4AB0010448C022070B588B0CF
:108FD000040004AD002604960922002105A8FDF72F
:108FE00057F800960922002101A8FDF751F84B23FC
:108FF0002B700D226946280000F066FA002304E079
:109000005A1D69468A5CE2540133072BF8DD08B02B
:1090100070BD000010B501000148F9F75FF910BDFF
:109020008E8E022000B583B00100044B00930B2309
:1090300000220348F9F729F903B000BDB0AD0010D4
:109040008E8E02200523CB56002B01DB934211D1DB
:10905000094B9C466044434258418000074BC0582E
:10906000097901238B40013B93401840434258410A
:10907000C0B270470020FCE70000D0AFB8850220E6
:1090800070B50A79202A19D8174B9C466044434290
:1090900058418000154BC45801239340013B497946
:1090A00049B2002910DB08002025AA1A914218DCD9
:1090B0008B401C4201D00120404270BD0C4B0D4A38
:1090C00040210D48FAF7AEFA2020801A002805DB6F
:1090D0001A0082401442F0D00138F7E701204042E4
:1090E000EBE701204042E8E70000D0AFB88502205E
:1090F000D0AD0010D4AE0010FCAD001070B505006E
:109100000C001600FFF79EFF002801D0002007E0AA
:109110001548FAF721FB831912339B005A5101308D
:10912000237983420FD92378617809021943A27801
:1091300012041143E3781B060B4342009A5A530B67
:10914000E9D19219E7E701229A401300013B074A4F
:10915000944665446A425541B340054AAD00A9585A
:109160000B43AB5070BDC04638AE00100000D0AF0E
:10917000B885022010B5054B9C46604443425841D7
:10918000800041180248F9F7A9F810BD0000D0AFDF
:10919000988E022010B582B00A4B9C466044434230
:1091A00058418400E31C084A009222000748F9F75E
:1091B0006CF8844202DC001B02B010BD012040426A
:1091C000FAE7C0460000D0AF4CAE0010988E0220E7
:1091D000F8B505000E00F9F729F80700310028005E
:1091E000FFF74EFF041E09DB020031002800FFF7E5
:1091F00085FF3800F9F726F82000F8BD0148FAF796
:10920000ABFAC04638AE001070B504000B790125EA
:109210009D40013D9540F9F709F80C4BE3185A427F
:10922000534199000A4A8A5829001140A94206D19F
:109230009B00AA4306495A50F9F704F870BD054B44
:10924000054A8A210548FAF7EDF9C0460000D0AF7B
:10925000B885022070AE0010C0AE0010FCAD00104A
:1092600010B50400F8F7E2FF0A4BE3185A425341E5
:109270009B00094A00219950002306E01F21194054
:109280001A0012329200115101331F2BF6D9F8F750
:10929000D9FF10BD0000D0AFB8850220F0B5CE4692
:1092A000474680B581464B005B18DB004B44DC33FE
:1092B0001B689C460027202417E0AE067B011E4356
:1092C0004B005B18DB004B44DC2080469844404652
:1092D00006601F261640B046E0263602404606438A
:1092E000D8331E60641B7F195209002C04D025005E
:1092F000052CE2D90525E0E74B005918C90049447F
:109300000800DC3063460360C0BCB946B046F0BD1F
:10931000F0B505AC25784C006418E4000419DC3481
:109320002468A446002D01D01F2614E0002612E078
:109330005401A0256D0525434C006418E400041970
:109340002700DC373D600D4D3543D8342560053BA3
:1093500005321F242240052BEAD89B0652011343F5
:109360004C006218D20082181500DC352B60034BCC
:109370001E43D832166063462B60F0BD80E00000CB
:10938000F0B58BB004000D00160002680121A94061
:109390008A430260002B35D069004919C900411881
:1093A0000A00C8321868106004325868106004322D
:1093B00098681060DB68DC310B6069004B19DB00DA
:1093C000D033E318802252011343802212061A6020
:1093D0001A60234BAB40A3602268281D01231F00A5
:1093E00087403A43226022682800083083401343B4
:1093F00023601F2216404919C9006418D83426601A
:109400000BB0F0BD1022002106A8FCF741FE80231E
:109410005B020693F8235B0207938023DB02089329
:10942000C0231B030893102206A902A8FCF736FEEE
:109430006B005B19DB00E3181A00C8320299116057
:10944000039A01921A00CC3201991160049A019298
:109450001A00D03201991160059ADC331A60ACE72A
:109460000101010110B583070AD00300032102E0C6
:1094700001330B4205D01A78002AF9D1181A10BD11
:10948000030019680C4A0D4C8A188A4322420FD1F6
:109490005968094A04338A188A43224208D1596814
:1094A000054A04338A188A432242F1D000E001338E
:1094B0001A78002AFBD1E1E7FFFEFEFE8080808063
:1094C000F8B5C0460000000001B40248844601BC63
:1094D000604700BF0503002001B40248844601BC78
:1094E000604700BF5102002001B40248844601BC1D
:1094F000604700BFDD03002001B40248844601BC80
:10950000604700BFDD03002001B40248844601BC6F
:10951000604700BF0901002001B40248844601BC35
:10952000604700BFDD01002001B40248844601BC51
:08953000604700BFC1000020EC
:10953800636861696E5F746F203C3D204E554D5FD6
:10954800444D415F4348414E4E454C530000000096
:10955800463A5C5069636F53444B5C5069636F5C77
:109568007069636F2D73646B5C7372635C727032C5
:109578005F636F6D6D6F6E5C686172647761726551
:109588005F646D615C696E636C7564652F68617298
:1095980064776172652F646D612E6800647265710D
:1095A800203C3D20445245515F464F524345000000
:1095B8004552525F554E4B4E4F574E5F4D534700E5
:1095C8004C4F4749435F414E414C595A45525F56AB
:1095D800315F3000434150545552455F5354415216
:1095E80054454400434150545552455F4552524FEB
:1095F8005200000053797374656D20636C6F636B60
:10960800206F66202575206B487A2063616E6E6F27
:10961800742062652065786163746C792061636881
:109628006965766564000000389600100CFF00003C
:10963800A0802060A0804060C7201D40C7001D405A
:109648004700404000C00B00589600100BFF000078
:10965800A0802060A08040601D40C6001D404600DC
:10966800404000C00A000000789600100BFF000080
:10967800A0802060A08040600040C40000404600F8
:10968800404000C00A000000989600100BFF000040
:10969800A0802060A08040600040C60000404600D6
:1096A800404000C00A0000006368616E6E656C5F30
:1096B800636F6E6669675F7365745F636861696E1F
:1096C8005F746F006368616E6E656C5F636F6E6672
:1096D80069675F7365745F647265710002030405EE
:1096E800060708090A0B0C0D0E0F1011121314159A
:1096F800161A1B1C68775F69735F636C61696D6517
:109708006428626974732C206269745F696E646589
:1097180078290000463A5C5069636F53444B5C50AB
:1097280069636F5C7069636F2D73646B5C737263DC
:109738005C7270325F636F6D6D6F6E5C68617264CE
:10974800776172655F636C61696D5C636C61696D9B
:109758002E63000068775F636C61696D5F636C6599
:10976800617200004E6F207370696E6C6F636B736B
:109778002061726520617661696C61626C650000C8
:1097880072742D3E616C61726D5F6964203D3D208D
:1097980069640000463A5C5069636F53444B5C50FF
:1097A80069636F5C7069636F2D73646B5C7372635C
:1097B8005C636F6D6D6F6E5C7069636F5F74696D0C
:1097C800655C74696D652E6300000000696420267D
:1097D80026206964203C3D20706F6F6C2D3E6865C3
:1097E80061702D3E6D61785F6E6F64657300000077
:1097F800256C6C642028686920253032782900009F
:109808006964202626206964203C3D2068656170D3
:109818002D3E6D61785F6E6F64657300463A5C50EB
:1098280069636F53444B5C5069636F5C7069636F25
:109838002D73646B5C7372635C636F6D6D6F6E5CCC
:109848007069636F5F7574696C5C696E636C75646D
:10985800652F7069636F2F7574696C2F7068656107
:10986800702E6800706172656E745F696400000034
:109878006368696C645F6964000000007061726508
:109888006E745F696420213D206368696C645F6958
:10989800640000002170685F636F6E7461696E73A5
:1098A8005F6E6F646528706F6F6C2D3E68656170C0
:1098B8002C2072657573655F6964290075735F7321
:1098C800696E63655F626F6F74203C3D20494E543A
:1098D80036345F4D41580000463A5C5069636F5317
:1098E800444B5C5069636F5C7069636F2D73646B84
:1098F8005C7372635C636F6D6D6F6E5C7069636FD0
:109908005F626173655C696E636C7564652F70690D
:10991800636F2F74797065732E68000072656D6FC0
:109928007665645F6964203D3D206E6578745F6983
:109938006400000063616C6C6261636B000000008E
:10994800706F6F6C2D3E616C61726D5F696E5F70D8
:10995800726F6772657373203D3D206D616B655F43
:109968007075626C69635F69642869645F686967B8
:10997800682C206E6578745F696429006964202604
:1099880026202170685F636F6E7461696E735F6E05
:109998006F646528686561702C206964290000007F
:1099A80064656661756C745F616C61726D5F706F20
:1099B8006F6C5F696E697469616C697A656428297E
:1099C80000000000616C61726D5F696420213D20B8
:1099D800706F6F6C2D3E616C61726D5F696E5F7048
:1099E800726F677265737300726300004174746507
:1099F8006D7074656420746F20736C656570206980
:109A08006E73696465206F6620616E206578636592
:109A18007074696F6E2068616E646C65723B207546
:109A2800736520627573795F776169742069662050
:109A3800796F75206D75737400000000616C617238
:109A48006D5F706F6F6C5F63616E63656C5F616C97
:109A580061726D007570646174655F75735F7369B9
:109A68006E63655F626F6F7400000000616C617205
:109A78006D5F706F6F6C5F616C61726D5F63616C5D
:109A88006C6261636B0000006765745F656E747279
:109A980079000000616C61726D5F706F6F6C5F6759
:109AA80065745F64656661756C7400006765745FF2
:109AB800656E7472795F69645F6869676800000041
:109AC80070685F667265655F6E6F646500000000B0
:109AD80070685F6164645F6368696C645F6E6F641B
:109AE8006500000070685F696E736572745F6E6F01
:109AF8006465000070685F6765745F6E6F64650019
:109B08006164645F616C61726D5F756E6465725FDC
:109B18006C6F636B00000000486172647761726566
:109B280020616C61726D20256420616C72656164CE
:109B38007920636C61696D656400000074696D6506
:109B4800725F68772D3E696E747320262031752008
:109B58003C3C20616C61726D5F6E756D00000000A9
:109B6800463A5C5069636F53444B5C5069636F5C61
:109B78007069636F2D73646B5C7372635C727032AF
:109B88005F636F6D6D6F6E5C68617264776172653B
:109B98005F74696D65725C74696D65722E6300002F
:109BA80068617264776172655F616C61726D5F7321
:109BB80065745F7461726765740000007570646134
:109BC80074655F75735F73696E63655F626F6F74E9
:109BD80000000000746F74616C000000463A5C502D
:109BE80069636F53444B5C5069636F5C7069636F62
:109BF8002D73646B5C7372635C636F6D6D6F6E5C09
:109C08007069636F5F73796E635C6D757465782EC8
:109C1800630000006D74782D3E636F72652E73705B
:109C2800696E5F6C6F636B006C6F636B5F69735F0A
:109C38006F776E65725F69645F76616C6964286DC1
:109C480074782D3E6F776E65722900006D74782DDB
:109C58003E656E7465725F636F756E740000000018
:109C68006D757465785F6578697400006D757465E5
:109C7800785F656E7465725F626C6F636B5F756E3B
:109C880074696C007570646174655F75735F73697E
:109C98006E63655F626F6F7400000000726F6F74AF
:109CA8005F696400463A5C5069636F53444B5C508B
:109CB80069636F5C7069636F2D73646B5C73726347
:109CC8005C636F6D6D6F6E5C7069636F5F757469EF
:109CD8006C5C70686561702E630000002170685FBD
:109CE8006765745F6E6F646528686561702C2072A3
:109CF8006F6F745F6964292D3E7369626C696E6762
:109D0800000000002170685F6765745F6E6F6465AE
:109D180028686561702C20726F6F745F6964292DE3
:109D28003E706172656E7400666F756E6400000047
:109D38006E65775F7375625F7472656520213D207B
:109D4800686561702D3E726F6F745F696400000012
:109D580070685F72656D6F76655F616E645F66726D
:109D680065655F6E6F64650070685F72656D6F76BC
:109D7800655F616E795F68656164000070685F6146
:109D880064645F6368696C645F6E6F64650000009B
:109D980070685F6765745F6E6F6465002C20667518
:109DA8006E6374696F6E3A2000000000617373651A
:109DB8007274696F6E2022257322206661696C6552
:109DC800643A2066696C6520222573222C206C6910
:109DD8006E65202564257325730A000031203D3DFA
:109DE800202875696E747074725F74296C2D3E73C7
:109DF80070696E5F6C6F636B00000000463A5C50E0
:109E080069636F53444B5C5069636F5C7069636F3F
:109E18002D73646B5C7372635C7270325F636F6D19
:109E28006D6F6E5C7069636F5F72756E74696D6576
:109E38005C72756E74696D652E6300000A2A2A2AA1
:109E48002050414E4943202A2A2A0A000A000000CD
:109E580072756E74696D655F696E697400000000E3
:109E68007372635F66726571203E3D20667265712C
:109E780000000000463A5C5069636F53444B5C50E5
:109E880069636F5C7069636F2D73646B5C73726375
:109E98005C7270325F636F6D6D6F6E5C6861726467
:109EA800776172655F636C6F636B735C636C6F6320
:109EB8006B732E6300000000636C6F636B5F636FEE
:109EC8006E6669677572650064656C7461203E3DF5
:109ED800202D323034382026262064656C746120A9
:109EE8003C3D203230343620262620212864656CFB
:109EF8007461202620312900463A5C5069636F530B
:109F0800444B5C5069636F5C7069636F2D73646B5D
:109F18005C7372635C7270325F636F6D6D6F6E5CE1
:109F280068617264776172655F6972715C69727188
:109F38002E630000212864656C7461203E3E203148
:109F48003175290063757272656E74203D3D205F1E
:109F58005F756E68616E646C65645F757365725F6A
:109F6800697271207C7C2063757272656E74203D05
:109F78003D2068616E646C65720000006972715FF3
:109F880068616E6465725F636861696E5F66726559
:109F9800655F736C6F745F68656164203E3D203057
:109FA80000000000767461626C655F68616E646CC5
:109FB8006572203D3D205F5F756E68616E646C65FB
:109FC800645F757365725F697271000021282828C3
:109FD8002875696E747074725F7429767461626C26
:109FE800655F68616E646C657229202D202828756C
:109FF800696E747074725F74296972715F68616EDA
:10A00800646C65725F636861696E5F736C6F7473AB
:10A0180029202D2031292573697A656F6628737484
:10A0280072756374206972715F68616E646C6572C1
:10A038005F636861696E5F736C6F74292900000043
:10A0480030783163203D3D20282A696E7374293E9B
:10A058003E313175000000002165786365707469D0
:10A068006F6E207C7C20657863657074696F6E20E4
:10A078003D3D206E756D202B2031360066616C7376
:10A088006500000069735F7368617265645F697277
:10A09800715F7261775F68616E646C657228736C5A
:10A0A8006F745F68616E646C6572290065786365BA
:10A0B8007074696F6E0000006972715F6164645F3B
:10A0C8007461696C5F746F5F667265655F6C6973F4
:10A0D80074000000696E736572745F6272616E630A
:10A0E800685F616E645F6C696E6B00006972715FB6
:10A0F80072656D6F76655F68616E646C657200008D
:10A108006D616B655F6272616E6368007265736F23
:10A118006C76655F6272616E636800006972715F78
:10A128007365745F6578636C75736976655F68617C
:10A138006E646C65720000006662646976203E3D5C
:10A14800203136202626206662646976203C3D2030
:10A1580033323000463A5C5069636F53444B5C506D
:10A1680069636F5C7069636F2D73646B5C73726392
:10A178005C7270325F636F6D6D6F6E5C6861726484
:10A18800776172655F706C6C5C706C6C2E6300003C
:10A1980028706F73745F64697631203E3D203120EA
:10A1A800262620706F73745F64697631203C3D20E9
:10A1B80037292026262028706F73745F64697632E9
:10A1C800203E3D203120262620706F73745F64691D
:10A1D8007632203C3D20372900000000706F7374F0
:10A1E8005F64697632203C3D20706F73745F6469E8
:10A1F800763100007265665F6D687A203C3D2028E4
:10A2080076636F5F66726571202F203136290000F2
:10A21800706C6C5F696E697400000000666E69009E
:10A22800666E692B000000006E616E00666E692D17
:10A23800000000008E4B00103E4B00103E4B0010FB
:10A24800984B00103E4B00103E4B00103E4B001048
:10A258003E4B00103E4B00103E4B00103E4B001092
:10A26800844B00103E4B00107A4B00103E4B001000
:10A278003E4B0010704B0010304C0010564C001034
:10A288006E4C0010564C0010104C0010564C00102C
:10A29800564C0010564C0010564C0010564C0010EE
:10A2A800564C0010564C00104C4C0010564C0010E8
:10A2B800564C0010564C0010564C0010564C0010CE
:10A2C8007A4C0010AA500010C0500010C050001066
:10A2D800C0500010C0500010C0500010C0500010F6
:10A2E800C0500010C0500010C0500010C0500010E6
:10A2F800C0500010C0500010C0500010C0500010D6
:10A30800C0500010C0500010C0500010C0500010C5
:10A31800C0500010C0500010C0500010C0500010B5
:10A32800C0500010C0500010C0500010C0500010A5
:10A33800C0500010C0500010C0500010C050001095
:10A34800C0500010D24E0010924E0010D24E001095
:10A35800C0500010C0500010C0500010C050001075
:10A36800C0500010C0500010C0500010C050001065
:10A37800C0500010C0500010C0500010C050001055
:10A38800C0500010C0500010C0500010C050001045
:10A39800864C0010C0500010C0500010C050001073
:10A3A800C0500010C0500010C0500010C050001025
:10A3B800C0500010C0500010864C0010224F0010F2
:10A3C800864C0010D24E0010924E0010D24E001053
:10A3D800C0500010864C0010C0500010C050001033
:10A3E800C0500010C0500010C0500010864C001023
:10A3F80074500010C0500010C05000109A4F001048
:10A40800C0500010864C0010C0500010C050001002
:10A41800864C001000000000000000000000F03F23
:10A428000000000000002440000000000000594027
:10A438000000000000408F40000000000088C3407A
:10A4480000000000006AF8400000000080842E41EF
:10A4580000000000D01263410000000084D797413B
:10A468000000000065CDCD412A282875696E743832
:10A478005F74202A29282828766F6964202A29727F
:10A488006F6D5F646174615F6C6F6F6B757028725C
:10A498006F6D5F7461626C655F636F6465282753D5
:10A4A800272C202746272929292D322929202A2007
:10A4B80034203E3D2053465F5441424C455F56325E
:10A4C8005F53495A45000000463A5C5069636F5330
:10A4D800444B5C5069636F5C7069636F2D73646B88
:10A4E8005C7372635C7270325F636F6D6D6F6E5C0C
:10A4F8007069636F5F646F75626C655C646F7562C9
:10A508006C655F696E69745F726F6D2E6300000021
:10A518005F5F61656162695F646F75626C655F69E1
:10A528006E6974002A282875696E74385F74202A49
:10A538002928726F6D5F7461626C652D322929203C
:10A548002A2034203E3D2053465F5441424C455F0B
:10A5580056325F53495A4500463A5C5069636F5317
:10A56800444B5C5069636F5C7069636F2D73646BF7
:10A578005C7372635C7270325F636F6D6D6F6E5C7B
:10A588007069636F5F666C6F61745C666C6F617431
:10A598005F696E69745F726F6D2E63005F5F6165DE
:10A5A8006162695F666C6F61745F696E69740000EF
:10A5B8004465627567000000626F6F74325F7732BE
:10A5C8003571303830000000302E3100312E332EF6
:10A5D800310000007069636F000000004C6F67690C
:10A5E80063416E616C797A65720000005365702072
:10A5F800203320323032320006005250BBFF3CB6C6
:10A60800DCA50010060052503ABCA911D0A50010D4
:10A6180006005250E182887FC0A500100600525003
:10A62800D3F07542B8A500106C656E203D3D203111
:10A6380000000000463A5C5069636F53444B5C501D
:10A6480069636F5C7069636F2D73646B5C737263AD
:10A658005C7270325F636F6D6D6F6E5C7069636F93
:10A668005F737464696F5C737464696F2E63000050
:10A678007570646174655F75735F73696E63655F38
:10A68800626F6F7400000000676574636861725FD1
:10A6980074696D656F75745F757300000D0A00004D
:10A6A800616400106564001071640010C1640010DA
:10A6B800A5640010000000005553422073746469BB
:10A6C8006E202F207374646F75740000060052505A
:10A6D80053B4F4A1C0A600107570646174655F7509
:10A6E800735F73696E63655F626F6F74000000006B
:10A6F80052617370626572727920506900000000BF
:10A708005069636F00000000426F61726420434427
:10A71800430000005265736574000000090254008C
:10A72800030100807D080B000202020000090400FA
:10A738000001020200040524002001052401000193
:10A7480004240202052406000107058103080010FD
:10A7580009040100020A0000000705020240000087
:10A76800070582024000000904020000FF000105FD
:10A7780012010002EF0201408A2E0A0000010102C4
:10A788000301000000000000F8A6001008A7001050
:10A798007C8E022010A700101CA7001028287569BD
:10A7A8006E747074725F7420296E6578745F627558
:10A7B800666665725F7074722026203062313131AE
:10A7C8003131317529203D3D20300000463A5C503A
:10A7D80069636F53444B5C5069636F5C7069636F66
:10A7E8002D73646B5C6C69625C74696E79757362F5
:10A7F8005C7372635C706F727461626C655C7261C9
:10A808007370626572727970695C7270323034305C
:10A818005C6463645F7270323034302E6300000011
:10A8280068775F646174615F6F6666736574286ECC
:10A838006578745F6275666665725F7074722920E8
:10A848003C3D205553425F445052414D5F4D415865
:10A8580000000000556E68616E646C6564204952A2
:10A868005120307825780A007268706F7274203D24
:10A878003D2030006463645F656470745F7866656A
:10A88800720000006463645F656470745F6F706574
:10A898006E0000006463645F7365745F6164647272
:10A8A800657373006463645F696E745F656E61628B
:10A8B8006C6500005F68775F656E64706F696E74C1
:10A8C8005F616C6C6F6300006463645F696E6974D8
:10A8D8000000000021286275665F6374726C202690
:10A8E800205553425F4255465F4354524C5F46558C
:10A8F8004C4C2900463A5C5069636F53444B5C509A
:10A9080069636F5C7069636F2D73646B5C6C6962FB
:10A918005C74696E797573625C7372635C706F7274
:10A928007461626C655C7261737062657272797071
:10A93800695C7270323034305C7270323034305F3F
:10A948007573622E630000006275665F6374726CD3
:10A958002026205553425F4255465F4354524C5F70
:10A9680046554C4C00000000657020256420257376
:10A978002077617320616C7265616479206176610A
:10A98800696C61626C6500005741524E3A207374DD
:10A99800617274696E67206E6577207472616E7378
:10A9A800666572206F6E20616C72656164792061E2
:10A9B80063746976652065702025642025730A0014
:10A9C80043616E277420636F6E74696E75652078B5
:10A9D800666572206F6E20696E61637469766520A2
:10A9E8006570202564202573000000006F757400D1
:10A9F800696E000073796E635F65705F6275666685
:10AA08006572000025732025643A2041535345524E
:10AA180054204641494C45440D0A0000607200101C
:10AA2800BE710010EE7100102A72001060720010E2
:10AA38006072001046720010EE7100106072001013
:10AA48006072001060720010607200106072001076
:10AA58006072001060720010D0710010E27A00106D
:10AA6800BC7A0010987C0010967A0010987C001030
:10AA7800FE7900108A7A0010987C00101A7A00106B
:10AA8800327A0010FE7C0010F07C0010427D00102D
:10AA9800B27E00102E7E00104E7E0010567D0010F3
:10AAA800A27D0010B67E0010757362645F656470E5
:10AAB800745F786665720000757362645F656470C0
:10AAC800745F6F70656E0000757362645F6F7065A8
:10AAD8006E5F656470745F70616972006F73616C3A
:10AAE8005F71756575655F73656E640070726F631D
:10AAF8006573735F6765745F6465736372697074A7
:10AB08006F72000070726F636573735F7365745F53
:10AB1800636F6E666967000070726F636573735F59
:10AB2800636F6E74726F6C5F7265717565737400B4
:10AB38007475645F7461736B0000000055830010C6
:10AB480011840010558400104D8500108186001076
:10AB580000000000757362645F636F6E74726F6CDF
:10AB68005F786665725F6362000000007475645FF9
:10AB7800636F6E74726F6C5F7866657200000000B8
:10AB8800636463645F786665725F636200000000F7
:10AB9800636463645F6F70656E0000007475645F62
:10ABA8006364635F6E5F77726974655F666C757303
:10ABB8006800000074755F656470745F76616C6925
:10ABC8006461746500000000747573625F696E6982
:10ABD800740000006C656E203E203000463A5C50E0
:10ABE80069636F53444B5C5069636F5C7069636F52
:10ABF8002D73646B5C7372635C7270325F636F6D2C
:10AC08006D6F6E5C7069636F5F756E697175655F96
:10AC180069645C756E697175655F69642E630000AF
:10AC28007069636F5F6765745F756E697175655F7D
:10AC3800626F6172645F69645F737472696E6700E2
:10AC4800666C6173685F6F666673202B20636F752F
:10AC58006E74203C3D205049434F5F464C41534859
:10AC68005F53495A455F425954455300463A5C5030
:10AC780069636F53444B5C5069636F5C7069636FC1
:10AC88002D73646B5C7372635C7270325F636F6D9B
:10AC98006D6F6E5C68617264776172655F666C6126
:10ACA80073685C666C6173682E630000636F6E6E18
:10ACB8006563745F696E7465726E616C5F666C6102
:10ACC800736820262620666C6173685F65786974EE
:10ACD8005F78697020262620666C6173685F7261F0
:10ACE8006E67655F657261736520262620666C61F4
:10ACF80073685F666C7573685F636163686500009D
:10AD0800636F6E6E6563745F696E7465726E616C95
:10AD18005F666C61736820262620666C6173685FC5
:10AD2800657869745F78697020262620666C61737F
:10AD3800685F72616E67655F70726F6772616D20C0
:10AD4800262620666C6173685F666C7573685F633E
:10AD58006163686500000000636F6E6E6563745F11
:10AD6800696E7465726E616C5F666C6173682026CB
:10AD78002620666C6173685F657869745F786970AE
:10AD880020262620666C6173685F666C7573685F41
:10AD98006361636865000000666C6173685F646F77
:10ADA8005F636D64000000004E6F20444D412063D6
:10ADB80068616E6E656C7320617265206176616989
:10ADC8006C61626C6500000070726F6772616D2D56
:10ADD8003E6C656E677468203C3D2050494F5F4962
:10ADE8004E535452554354494F4E5F434F554E545A
:10ADF80000000000463A5C5069636F53444B5C5056
:10AE080069636F5C7069636F2D73646B5C737263E5
:10AE18005C7270325F636F6D6D6F6E5C68617264D7
:10AE2800776172655F70696F5C70696F2E6300008F
:10AE38004E6F2070726F6772616D20737061636509
:10AE4800000000004E6F2050494F207374617465F4
:10AE5800206D616368696E65732061726520617633
:10AE680061696C61626C650070726F6772616D5FB9
:10AE78006D61736B203D3D20285F757365645F6964
:10AE88006E737472756374696F6E5F7370616365F6
:10AE98005B70696F5F6765745F696E646578287059
:10AEA800696F295D20262070726F6772616D5F6D12
:10AEB80061736B290000000070696F5F72656D6FC8
:10AEC80076655F70726F6772616D00005F70696FA1
:10AED8005F66696E645F6F66667365745F666F72DE
:0CAEE8005F70726F6772616D0000000007
:10AEF400B4020010A80200109C02001000A600106A
:10AF0400900200100CA6001018A6001024A6001031
:04AF1400D4A60010AF
:10AF180010B5D0231B0600241C570268EFF31081DC
:10AF280072B61368002BFCD0BFF35F8F0423C3569F
:10AF3800002B08DB0368BFF35F8F00221A6081F3E0
:10AF4800108820BFE9E704710368BFF35F8F002210
:10AF58001A6081F3108810BD03000068EFF3108CAD
:10AF680072B60268002AFCD0BFF35F8F04229A569B
:10AF7800002A0BDB002910D00A6000201B68BFF3F1
:10AF88005F8F00221A608CF310887047D022120657
:10AF9800127852B21A710120F0E70020EEE70000A3
:10AFA800F8B5CE46474680B50400170098460368B2
:10AFB800002B20D0D0231B061B785BB2994626684D
:10AFC800EFF3108C72B63568002DFCD0BFF35F8F9D
:10AFD80004256557002D14DB2368BFF35F8F00221B
:10AFE8001A608CF310883800414600F039F90028BF
:10AFF800E5D000200FE00A4B0A4A7A210A4800F0FF
:10B0080017F94B4623712368BFF35F8F00221A603C
:10B018008CF310880120C0BCB946B046F8BDC046C4
:10B028001C9C0010749C0010E49B0010F0B5C646F0
:10B0380000B582B00700884600F002F904000D1E32
:10B048001CDB0190FA22920000234046002100F008
:10B05800FFF822002B0012184B419D4202D804D160
:10B06800944202D901225242D317002B0CDB38003C
:10B07800FFF796FF02B080BCB846F0BD054B064A04
:10B088003F21064800F0D4F8024B034A3F21034809
:10B0980000F0CEF8C49800108C9C0010E0980010C6
:10B0A80010B50268EFF3108172B61368002BFCD05C
:10B0B800BFF35F8F0423C356002B0ADBFF23037102
:10B0C8000368BFF35F8F00221A6081F3108840BFC6
:10B0D80010BD034B034AA921034800F0A9F8C04654
:10B0E800309C0010689C0010E49B0010094B1B78F2
:10B0F800002B08D00CE09A008021490551180868F7
:10B108000549505001333F2BF5DD024B01221A70DF
:10B118007047C046928E0220D085022010B5024B9F
:10B128000133984710BDC046D085022000280AD0B8
:10B1380003231B02054A12685340C02292001340A1
:10B14800034A136070470223F3E7C0460C800140AE
:10B158000C900140F0B5D6464F464646C0B50700AC
:10B168000E00150018239A461B8814229046108852
:10B1780028499847814653461B88424610882649E5
:10B188009847040053461B8842461088234998472D
:10B1980080464B46002B0CD0002C0AD0002808D043
:10B1A800FFF7A4FFC847A0470020FFF7BFFF2A000A
:10B1B8000FE01B4B1B4A80211B4800F039F8002B7D
:10B1C80007D0002A05D0C0235B051B6E3370013AF7
:10B1D80001362B00134312D0C0235B059C6A082359
:10B1E8002340A107EBD5002DE9D0511B0D29E6D846
:10B1F8003878C02149050866013D0137DFE701209D
:10B20800FFF794FFC047FFF789FFE0BCBA46B14695
:10B21800A846F0BD494600004558000046430000D6
:10B2280060AD0010A0AD001074AC00107047C046AF
:10B2380001B40248844601BC604700BF25360010AF
:10B2480001B40248844601BC604700BF492F001082
:10B2580001B40248844601BC604700BF655E001027
:10B2680001B40248844601BC604700BF252E001087
:10B278002804002009FF0000A080206000E007C02B
:10B28800E0A04460A40001E008000000248102203E
:10B29800200010005C040020000000000080022054
:10B2A800048702200000000000000000148702202C
:10B2B8000000000000000000100000000000000076
:10B2C8000000010000000000000000000000020073
:10B2D8000000000000000000000003000000000063
:10B2E800000000000000FF000000000000B54868F2
:10B2F80001318E460047704609380149884700BD2C
:10B30800AD3C00100000000000000000000000003C
:10B31800503300004C330000543300005233000017
:10B328004D5300004D4300005334000043340000E7
:10B33800E1650010000000005165001000000000E9
:10B3480000010000F4A90010F8A90010F8840220F8
:10B3580010000C000000E0FF1F00000000000000CB
:10B3680000000000000000000000000000000000D5
:10B3780000000000000000000000000000000000C5
:10B38800816000102551001035580010515F0010E1
:08B39800ED0200105D8F0010B2
:04000005100001E9FD
:00000001FF
